:1000000016C3000033C3000031C300002FC300003B
:100010002DC300002BC3000029C3000027C300002C
:1000200025C3000023C3000021C300001FC300003C
:100030000C94933F1BC3000019C3000017C30000BA
:1000400015C3000013C300000C947F3F0FC30000D2
:100050000DC300000BC3000009C3000007C300006C
:1000600005C3000003C3000001C30000FFC200007D
:10007000FDC20000FBC20000F9C20000F7C2000090
:10008000F5C20000F3C20000F1C20000180A1D0A08
:100090002B0A300A350A3A0A3F0A440AD20DD70D14
:1000A000E50DEA0DEF0DF40DF90DFE0DF512F81248
:1000B000FB12FE120113041307130A13441F691FD6
:1000C0007D1F901F931FA41FB51FD31F5A1F5D1FB5
:1000D000C61FC91FCC1F601F631F661FF9240F2591
:1000E00023253B25512567258B25A125B72582276B
:1000F000EF271C298729AF2AE42BD22CD02D082FDB
:10010000592FC32F0E3018307930D430D730DA3031
:10011000DD30E030E330E630E9309B33B133C733D4
:10012000DE33F4330A34203436348A348D34903458
:100130009334963499349C349F34F7347335EF35C7
:10014000783601377837F4375E38C8384139AE39F8
:10015000253AAB3A2E3B00000000000000000404EA
:100160000404000400000A0A0A00000000000A0A51
:100170001F0A1F0A0A00040F140E051E0400181996
:100180000204081303000C12140814120D000C04CE
:100190000800000000000204080808040200080427
:1001A0000202020408000004150E150400000004F9
:1001B000041F04040000000000000C0408000000FC
:1001C000001F0000000000000000000C0C000001F7
:1001D0000204081000000E11131519110E00040C72
:1001E000040404040E000E11010204081F001F0283
:1001F000040201110E0002060A121F0202001F1063
:100200001E0101110E000608101E11110E001F0123
:100210000204080808000E11110E11110E000E1133
:10022000110F01020C000001020408100000000C74
:100230000C000C040800020408100804020000006E
:100240001F001F00000008040201020408000E1134
:100250000102040004000E11010D15150E000E110F
:1002600011111F1111001E11111E11111E000E116E
:10027000101010110E001C12111111121C001F1071
:10028000101E10101F001F10101E101010000E1155
:10029000101711110E001111111F111111000E0470
:1002A000040404040E000702020202120C001112E0
:1002B0001418141211001010101010101F00111B30
:1002C00015151111110011111915131111000E112D
:1002D000111111110E001E11111E101010000E111F
:1002E000111115120D001E11111E141211000F1004
:1002F000100E01011E001F04040404040400111167
:10030000111111110E0011111111110A0400111116
:10031000111115150E0011110A040A111100111105
:10032000110A040404001F01020408101F000E0833
:10033000080808080E00110A1F041F0404000E021A
:10034000020202020E00040A110000000000000078
:10035000000000001F000804000000000000000072
:100360000E010F110F0010101E1111111E000000C0
:100370000E1010110E0001010D1311110F000000DD
:100380000E111F100E000609081C08080800000FB7
:1003900011110F010E001010161911111100040097
:1003A0000C0404040E000200060202120C001010DD
:1003B0001214181412001808080808081C0000007D
:1003C0001A15151111000000161911111100000065
:1003D0000E1111110E0000001E111E101000000061
:1003E0000F110F010100000016191010100000007D
:1003F0000E100E011E0008081C0808090600000067
:10040000111111130D0000001111110A0400000058
:10041000111111150A000000110A040A1100000050
:1004200011110F010E0000001F0204081F003844C4
:1004300044447C4444007C40407844447800784400
:100440004478444478007C404040404040000C14D4
:10045000242424243C447C40407840407C00545474
:100460005438545454003844041804443800444464
:100470004C546444440054444C5464444400444840
:100480005060504844001C24242424246400446CFC
:100490005454444444004444447C44444400384458
:1004A0004444444438007C44444444444400784434
:1004B00044784040400038444040404438007C107C
:1004C0001010101010004444443C044438003854C8
:1004D0005454381010004444281028444400444424
:1004E000444444447E02444444443C040400545480
:1004F000545454547C005454545454547E02602038
:100500002038242438004444446454546400404057
:100510004078444478003844041C0444380048546B
:100520005474545448003C44443C14244400000097
:1005300038043C443C0000007840784478000000D7
:10054000784C784C78000000784040404000000033
:10055000182828287C44000038447C403C000000D7
:1005600054543854540000007804380478000000D3
:10057000444C546444000010444C54644400000053
:1005800044487048440000001C24444444000000D7
:10059000446C545444000000484878484800000027
:1005A0003844444438000000784848484800000077
:1005B0007048704040000000384040403800000063
:1005C0007C1010101000000048483808700000002F
:1005D000385454381000000044281028440000000B
:1005E000484848487C040000484838080800000093
:1005F000545454547C000000545454547E0200005F
:1006000060203C223C0000004242724A720000001E
:1006100040407844780000007008780870000000BE
:100620004C5272524C0000003C443C4444001124A3
:100630001FBECFEFD0E1DEBFCDBF15E0A0E0B1E03F
:10064000E4E0F0E900E00BBF02C007900D92A63E87
:10065000B107D9F726E0A6EEB5E001C01D92A23A97
:10066000B207E1F70E94F13F0C940048C9CCE2E6E2
:10067000F0E090819E7F9083908194609083908140
:10068000977F9083A8988BBB8DE08A95F1F7000047
:10069000A89A8081886080830895E2E6F0E09081E6
:1006A000916090839081946090839081977F9083F4
:1006B000A8988BBB8DE08A95F1F70000A89A8081FD
:1006C000886080830895CF93C82F892FE6DF8C2F11
:1006D000CF91E3CFE2E6F0E020812160208320810A
:1006E000246020832081277F2083A8988BBB92BB26
:1006F0008DE08A95F1F70000A89A80818860808358
:100700000895CF93C82F86E3B2DFC13049F030F0AF
:10071000C23041F0C33059F488EE07C088E403C00A
:1007200088E203C088E8B9DF04C0B7DF0BC0CD7F23
:1007300049F48FEE90E09093E9058093E8058FE30C
:1007400091E008C08FE391E09093E9058093E8057C
:100750008FEE90E09093E7058093E605CF910895A2
:10076000CF93C82F8FEF8ABB81BB8093610081E05C
:1007700084BBE2E6F0E080818260808381E077DF05
:100780002FEF89E698E1215080409040E1F700C0CA
:10079000000080EC6CDF85E280DF81EC68DF81E1C6
:1007A0007CDF85EC64DF8BE278DF8BE276DF87EC41
:1007B0005EDF86E872DF8C2FA4DF8AE358DF85E0F6
:1007C0006CDF81EB54DF80E068DF88E166DF86EB79
:1007D0004EDF8AE062DF82E860DF87E25EDF81E190
:1007E00046DF2FEF8DEE92E0215080409040E1F700
:1007F00000C0000089E2CF913ACF0F931F93CF93AF
:10080000DF938C01EB018AE232DFC8015CDFCE01AD
:10081000DF91CF911F910F9156CF0F931F93CF93DD
:10082000DF938C01EB018BE222DFC8014CDFCE01AC
:10083000DF91CF911F910F9146CFCF93DF93EB01C3
:10084000BC01DBDFBE01CE01E8DF8CE2DF91CF919E
:100850000ECFCF93DF93EA01F0DFCE01DF91CF918E
:1008600039CF8F929F92AF92BF92CF92DF92EF9249
:10087000FF920F931F93CF93DF93A8956817790783
:1008800038F4862797276827792786279727A895FA
:100890002417350738F442275327242735274227C2
:1008A0005327A895A091E805B091E905FC01A81788
:1008B000B90708F4FD016B01A617B70708F46D012D
:1008C0008091E6059091E705EA018417950708F401
:1008D000EC0179018217930708F47C01A895960131
:1008E0002F5F3F4F2E1B3F0BD7011196AC1BBD0B4B
:1008F0000E94C8444B015C01B601CF017EDFA89580
:10090000B701CE018ADF8CE2B2DEA895C12CD12CD2
:100910007601C814D904EA04FB0449F0C801DADE00
:10092000A8958FEFC81AD80AE80AF80AF2CFDF9123
:10093000CF911F910F91FF90EF90DF90CF90BF90DC
:10094000AF909F908F9008950F931F93411551057D
:1009500079F02115310561F0FA01AB01615071099F
:10096000260F371FBC01615071096E0F7F1F79DFA1
:100970001F910F9108952F923F924F925F926F9225
:100980007F928F929F92AF92BF92CF92DF92EF921F
:10099000FF920F931F93CF93DF93CDB7DEB7679787
:1009A0000FB6F894DEBF0FBECDBF5C01798B688BAC
:1009B000598748873B872A870F83F12C28E0029FBD
:1009C000C00111241A821982E8E0F0E0FF8BEE8B5F
:1009D00047019C01285F31093B8B2A8BFC01E052C7
:1009E000F340FD8BEC8BC888D98889819A81C80E29
:1009F000D91E8A899B89EE89FF898E1B9F0B9C01DA
:100A00002A5A3E4F3F872E878C899D898E1B9F0BCC
:100A1000FC01EA5AFE4FFD87EC871E821D821C8274
:100A20001B8287E0682E712C412C512C212C312CFB
:100A3000FF81F7FD1EC0EE85FF85849190E0062CB6
:100A400002C0959587950A94E2F780FF08C0088553
:100A500019859701A701B6018D819E8107C00A857E
:100A60001B859701A701B6018B819C818A0D9B1D77
:100A700020C0FF81F03CF0F0EC85FD85849190E092
:100A8000062C02C0959587950A94E2F780FF09C06D
:100A9000088519859701A701B601C501820D931D2F
:100AA00008C00A851B859701A701B601C501840D01
:100AB000951D4ADF280C391C480C591CF1E06F1AAF
:100AC00071082B813C81280D391D3C832B838D813E
:100AD0009E81880D991D9E838D839FEF69167906EF
:100AE00009F0A6CFEE89FF893197FF8BEE8B298124
:100AF0003A812E0D3F1D3A832983EF2B09F073CFE6
:100B000067960FB6F894DEBF0FBECDBFDF91CF91D1
:100B10001F910F91FF90EF90DF90CF90BF90AF901B
:100B20009F908F907F906F905F904F903F902F900D
:100B300008954F925F926F927F928F929F92AF92A1
:100B4000BF92CF92DF92EF92FF920F931F93CF93BA
:100B5000DF93EC016B014A013901102F88E0089FF7
:100B6000500111242701F20101912F010023B1F05E
:100B70002091E8053091E905CE010896281739073C
:100B800020F4CA0CDB1CC1E0D0E0E12E9301A401EB
:100B9000B601CE01F0DECA0DDB1DE5CFDF91CF91AE
:100BA0001F910F91FF90EF90DF90CF90BF90AF908B
:100BB0009F908F907F906F905F904F9008956F926D
:100BC0007F928F929F92AF92BF92CF92DF92EF92DD
:100BD000FF920F93CF93DF9300D000D0CDB7DEB755
:100BE0006C015B014A013901C70119821A821B821B
:100BF0001C824AE0BE016F5F7F4F0E94D744CE0146
:100C000001967C019301A401B501C60192DF0F900A
:100C10000F900F900F90DF91CF910F91FF90EF9079
:100C2000DF90CF90BF90AF909F908F907F906F900C
:100C300008950F931F932091E6053091E705609189
:100C4000E8057091E9058C0140E050E080E090E01B
:100C500008DE1F910F910895EF92FF920F931F935B
:100C6000CF93DF93EB018A017901BC01640F751FFB
:100C7000C4DDBE01CE01D1DD8CE2F9DCC0E0D0E004
:100C8000C017D10721F0C70125DD2196F9CFDF91EB
:100C9000CF911F910F91FF90EF900895EF92FF92E7
:100CA0000F931F93CF93DF93EB018A017901BC016E
:100CB000A4DDBE01600F711FCE01AFDD8CE2D7DC79
:100CC000C0E0D0E0C017D10721F0C70103DD2196B5
:100CD000F9CFDF91CF911F910F91FF90EF90089581
:100CE0002F923F924F925F926F927F928F929F923C
:100CF000AF92BF92CF92DF92EF92FF920F931F932A
:100D0000CF93DF9300D000D000D0CDB7DEB76C0119
:100D10007B015A0139012801261B370B3A832983AD
:100D20008A01081B190B17FF03C0119501951109C2
:100D3000CA14DB0420F022242A94322C03C022247B
:100D40002394312C89819A819E838D8397FF05C0DE
:100D50009195819591099E838D832D813E81319559
:100D6000219531093C832B83E614F70428F08FEF9B
:100D70009FEF9A83898304C021E030E03A8329837E
:100D800048018D819E81881A990AA201B701C60186
:100D900060DDC401880F991F2B813C818217930766
:100DA00064F0CA14DB0499F02D813E81821A930A03
:100DB000C20CD31C0817190744F3E614F70439F0E2
:100DC000800E911E89819A81E80EF91EDECF26964B
:100DD0000FB6F894DEBF0FBECDBFDF91CF911F914C
:100DE0000F91FF90EF90DF90CF90BF90AF909F90CA
:100DF0008F907F906F905F904F903F902F900895CD
:100E0000AF92BF92CF92DF92EF92FF920F931F9318
:100E1000CF93DF937C016B01EA01590198011CDF3C
:100E2000B501615071096C0D7D1D9801AE01C701BE
:100E300013DF9801A501B601C70130DFCE0101978C
:100E40009801A501B6018E0D9F1DDF91CF911F91D5
:100E50000F91FF90EF90DF90CF90BF90AF901ECF9B
:100E60002F923F924F925F926F927F928F929F92BA
:100E7000AF92BF92CF92DF92EF92FF920F931F93A8
:100E8000CF93DF931C012B01690150E0002711274C
:100E9000041B150BC1E0D0E0C41BD50BCC0FDD1F2C
:100EA000E12CF12CA6015701A40CB51CB5013101B0
:100EB000601A710AC301CDDCA601B5014801820C9C
:100EC000931CC401C6DCA6015201AE18BF08B501CF
:100ED000C401BFDCA601B501C301BBDCEC16FD06F5
:100EE000B4F08FEFE81AF80AC701880F991F01962E
:100EF0008C0F9D1F22273327201B310BE216F30690
:100F000039F40C171D074CF0C0E0D0E001C0CE0151
:100F10000C171D0714F0EC01C5CF0F5F1F4F980190
:100F2000220F331F2F5F3F4F820F931F10161106A2
:100F300094F7DF91CF911F910F91FF90EF90DF9089
:100F4000CF90BF90AF909F908F907F906F905F9069
:100F50004F903F902F9008954F925F926F927F92A3
:100F60008F929F92AF92BF92CF92DF92EF92FF92B9
:100F70000F931F93CF93DF93EC015B014A0139017B
:100F800028018601ADDE9701A201B301C401A8DEEC
:100F90009501AE01B701C201A3DEDF91CF911F9190
:100FA0000F91FF90EF90DF90CF90BF90AF909F9008
:100FB0008F907F906F905F904F900895CF93C82F40
:100FC0008A3011F48DE0FADF5D9BFECFCCB980E072
:100FD00090E0CF910895CF92DF92EF92FF920F931E
:100FE0001F93A8950FEF1FEF21E430E04FE550E08D
:100FF00065E070E085E090E003DFA89521E430E053
:101000004FE550E06BE470E085E090E0F9DE2BE422
:1010100030E04FE550E061E970E085E090E0F0DE1F
:10102000A3E3EA2EA5E0FA2E01E02FE130E04FEF36
:101030005FEF60E570E082E190E07BDDBEE2EB2EE9
:10104000B5E0FB2E2FE130E04FEF5FEF6AE570E097
:1010500083E290E06EDD0FEF1FEF21E430E04FE51B
:1010600050E065E070E08CED90E0CADE21E430E015
:101070004FE550E06BE470E08CED90E0C1DE2BE4D6
:1010800030E04FE550E061E970E08CED90E0B8DED3
:1010900013E3E12E15E0F12E01E02FE130E04FEFF8
:1010A0005FEF60E570E08BEE90E043DD88E2E82ED4
:1010B00085E0F82E2FE130E04FEF5FEF6AE570E05A
:1010C0008CEF90E036DD99E5E92E92E0F92E2FE1E4
:1010D00030E04FEF5FEF66EE70E08AE090E029DDF0
:1010E000A89580912A0690912B06019709F04FC090
:1010F0000FE110E024E430E048E550E064E970E0FE
:1011000088E090E021DC2CE430E04EE650E06CE832
:1011100070E089E690E018DC24E430E048E550E037
:1011200064E970E080EE90E00FDC20EE37E048E20A
:1011300064EB70E080EA90E093DE20EE37E047E277
:1011400064EB70E080EA90E08BDE20EE37E04BE26B
:1011500064EB70E080EA90E083DE20EE37E045E269
:1011600064EB70E080EA90E07BDEE0EECE2EE7E01C
:10117000DE2EF4EBEF2EF12C07EB10E028EC30E044
:1011800044E950E060EA70E084E990E0E5DEA8958B
:1011900080912A0690912B06892B09F051C00FE10E
:1011A00010E024E430E048E550E064E970E088E0D5
:1011B00090E0CADB2CE430E04EE650E06CE870E0F2
:1011C00089E690E0C1DB24E430E048E550E064E9E2
:1011D00070E080EE90E0B8DB20E038EF48E264EBAE
:1011E00070E080EA90E03CDE20E038EF47E264EB1C
:1011F00070E080EA90E034DE20E038EF4BE264EB10
:1012000070E080EA90E02CDE20E038EF45E264EB0D
:1012100070E080EA90E024DE00E018EF23E230E0A6
:1012200045E050E065EA70E086E990E08DDB23E27E
:1012300030E045E050E065EA70E085EA90E084DB6C
:10124000A89580912C0690912D06892B79F4A8956C
:101250007EE1E72E75E0F72E01E02FE130E04FEF61
:101260005FEF63E270E08AE090E063DC80912C063F
:1012700090912D060197E1F4A89557EDE52E55E0E4
:10128000F52E01E02FE130E04FEF5FEF64E170E019
:1012900084E190E04EDC61EDE62E65E0F62E2FE174
:1012A00030E04FEF5FEF68E270E08EE190E041DC0C
:1012B000A89580912C0690912D060297E1F4A895AF
:1012C0003AECE32E35E0F32E01E02FE130E04FEF72
:1012D0005FEF64E170E084E190E02BDC41EDE42E0F
:1012E00045E0F42E2FE130E04FEF5FEF68E270E071
:1012F0008EE190E01EDCA89580912C0690912D0641
:10130000039779F4A89523ECE22E25E0F22E01E074
:101310002FE130E04FEF5FEF63E270E089E190E0B2
:1013200008DCA89580912C0690912D06049779F4FD
:10133000A89594EEE92E94E0F92E01E02FE130E03B
:101340004FEF5FEF63E270E08FE090E0F2DBA89593
:1013500080912C0690912D060597E1F4A8950EED4D
:10136000E02E04E0F02E01E02FE130E04FEF5FEFE0
:1013700064E170E089E190E0DCDB84EDE82E84E05C
:10138000F82E2FE130E04FEF5FEF63E270E08FE087
:1013900090E0CFDBA89580912C0690912D060697C2
:1013A000E1F4A895BEEDEB2EB4E0FB2E01E02FE1B9
:1013B00030E04FEF5FEF64E170E089E190E0B9DB8E
:1013C00012ECE12E14E0F12E2FE130E04FEF5FEF51
:1013D00063E270E08FE190E0ACDBA89580912C0691
:1013E00090912D06079779F4A895A9EAEA2EA4E032
:1013F000FA2E01E02FE130E04FEF5FEF63E270E0A3
:101400008FE090E096DB80912C0690912D06892B41
:1014100009F048C0A895E09189068E2F90E08830A9
:10142000910508F03FC0FC01EA5BFF4F0C94BF44FC
:10143000F4EAEF2EF4E0FF2E04C0EFE9EE2EE4E034
:10144000FE2E02E02FE130E04FEF5FEF6EE170E043
:101450008BEE90E026C075E9E72E74E0F72E18C0F9
:101460006BE8E62E64E0F62E13C051E8E52E54E05A
:10147000F52E0EC047E7E42E44E0F42E09C03DE609
:10148000E32E34E0F32E04C023E6E22E24E0F22E15
:1014900001E02FE130E04FEF5FEF6EE170E086EEAC
:1014A00090E047DB80912C0690912D06019701F585
:1014B000A89580913506813069F038F08230C1F40A
:1014C00001E8E02E04E0F02E09C095E9E92E94E051
:1014D000F92E04C08BE8E82E84E0F82E01E02FE11D
:1014E00030E04FEF5FEF6EE170E086EE90E021DBE1
:1014F00080912C0690912D06029701F5A895809178
:101500003C06813069F038F08230C1F4A1E8EA2E5F
:10151000A4E0FA2E09C015E9E12E14E0F12E04C072
:10152000BBE8EB2EB4E0FB2E01E02FE130E04FEF03
:101530005FEF6EE170E086EE90E0FBDA80912C06C2
:1015400090912D06039779F4A895FFEEEF2EF4E025
:10155000FF2E01E02FE130E04FEF5FEF6EE170E032
:101560008EEE90E0E6DA80912C0690912D0604979D
:1015700001F5A89580919406813069F038F08230A9
:10158000C1F461E8E62E64E0F62E09C0E5E9EE2E2E
:10159000E4E0FE2E04C07BE8E72E74E0F72E01E0C5
:1015A0002FE130E04FEF5FEF6EE170E086EE90E00C
:1015B000C0DA80912C0690912D06059701F5A8952B
:1015C00080918806813069F038F08230C1F431E8CA
:1015D000E32E34E0F32E09C055E9E52E54E0F52E54
:1015E00004C04BE8E42E44E0F42E01E02FE130E0AB
:1015F0004FEF5FEF6EE170E086EE90E09ADA809157
:101600002C0690912D06069701F5A89580918506E8
:10161000813069F038F08230C1F481E8E82E84E04E
:10162000F82E09C025E9E22E24E0F22E04C09BE842
:10163000E92E94E0F92E01E02FE130E04FEF5FEF6B
:101640006EE170E086EE90E074DA80912C06909165
:101650002D06079709F4A8951F910F91FF90EF9021
:10166000DF90CF900895CF92DF92EF92FF920F9389
:101670001F93A89500EE17E021E430E048EC50E01D
:101680006AEA70E085E090E05FD90FEF1FEF21E498
:1016900030E048EC50E063E270E085E090E0B0DBE1
:1016A00087E7E82E82E0F82E01E02FE130E040EEFF
:1016B00057E06CE370E088E290E03BDA0FEF1FEF59
:1016C00020E530E040E550E065E070E08BEE90E032
:1016D00097DB90EEC92E97E0D92E24E1E22EF12C73
:1016E00003E111E026E430E041E351E066E470E01C
:1016F00085EF90E031DC37E1E32EF12C24E430E09B
:101700004FE251E064E470E087EF90E025DC0FEFFA
:101710001FEF20E530E040E550E064E670E08BEE3E
:1017200090E06EDB45EAE42EF12C03E111E023E7C3
:1017300030E041E351E063E770E085EF90E00CDCDE
:1017400053EAE52EF12C25E730E04FE251E065E762
:1017500070E087EF90E000DC66E4E62E65E0F62EB0
:1017600002E020EE37E040E050E068EC70E08DE20F
:1017700090E0DFD91F910F91FF90EF90DF90CF9015
:101780000895CF92DF92EF92FF920F931F93A89547
:1017900000EE17E021E430E048EC50E06AEA70E047
:1017A00085E090E0D1D80FEF1FEF21E430E048EC66
:1017B00050E063E270E085E090E022DB83EBE82E0E
:1017C00084E0F82E01E02FE130E040EE57E06CE3DA
:1017D00070E088E290E0ADD90FEF1FEF20E530E038
:1017E00040E550E065E070E08BEE90E009DB90EEC4
:1017F000C92E97E0D92E24E1E22EF12C03E111E06D
:1018000026E430E041E351E066E470E085EF90E0EB
:10181000A3DB37E1E32EF12C24E430E04FE251E08A
:1018200064E470E087EF90E097DB0FEF1FEF20E5B7
:1018300030E040E550E064E670E08BEE90E0E0DA06
:1018400045EAE42EF12C03E111E023E730E041E327
:1018500051E063E770E085EF90E07EDB53EAE52E30
:10186000F12C25E730E04FE251E065E770E087EFCB
:1018700090E072DB6FEDE62E65E0F62E02E020EEE2
:1018800037E040E050E068EC70E08DE290E051D944
:101890001F910F91FF90EF90DF90CF900895CF921E
:1018A000DF92EF92FF920F931F93A89500EE17E03F
:1018B00021E430E048EC50E06AEA70E085E090E036
:1018C00043D80FEF1FEF21E430E048EC50E063E233
:1018D00070E085E090E094DA82E5E82E84E0F82E6E
:1018E00001E02FE130E040EE57E06CE370E088E289
:1018F00090E01FD90FEF1FEF20E530E040E550E00A
:1019000065E070E08BEE90E07BDA90EEC92E97E018
:10191000D92E24E1E22EF12C03E111E026E430E09F
:1019200041E351E066E470E085EF90E015DB37E1DC
:10193000E32EF12C24E430E04FE251E064E470E067
:1019400087EF90E009DB0FEF1FEF20E530E040E587
:1019500050E064E670E08BEE90E052DA45EAE42E67
:10196000F12C03E111E023E730E041E351E063E7CC
:1019700070E085EF90E0F0DA53EAE52EF12C25E7F0
:1019800030E04FE251E065E770E087EF90E0E4DAA5
:1019900067E5E62E65E0F62E02E020EE37E040E057
:1019A00050E068EC70E08DE290E0C3D81F910F9199
:1019B000FF90EF90DF90CF900895CF93DF9300D00A
:1019C00000D0CDB7DEB7809163001C821B821A82E3
:1019D0001982BE016F5F7F4FCE0103960E942243A2
:1019E0008B819C818431954068F489819A81843A05
:1019F000964040F489819A818D32914018F082E0BE
:101A0000809352068B819C818937954090F08B8121
:101A10009C81843C994068F489819A81843A9640FB
:101A200040F489819A818D32914018F083E080934F
:101A300052068B819C8189329A4068F089819A8113
:101A400084379E4040F489819A81813D974018F007
:101A500081E0809352068B819C81863F994060F49F
:101A60008B819C818134964038F089819A81813DB7
:101A7000974010F010925206809152060F900F90EE
:101A80000F900F90DF91CF910895CF92DF92EF9258
:101A9000FF920F931F93A89500EE17E021E430E02A
:101AA00048EC50E06AEA70E085E090E00E94A4040F
:101AB0000FEF1FEF21E430E048EC50E063E270E00C
:101AC00085E090E09DD920E530E040E550E065E01C
:101AD00070E08BEE90E094D9F0EECF2EF7E0DF2EA1
:101AE000A4E1EA2EF12C03E111E026E430E041E329
:101AF00051E066E470E085EF90E02EDAB7E1EB2E7E
:101B0000F12C24E430E04FE251E064E470E087EF30
:101B100090E022DA0FEF1FEF20E530E040E550E0E3
:101B200064E670E08BEE90E06BD915EAE12EF12CC3
:101B300003E111E023E730E041E351E063E770E0C7
:101B400085EF90E009DA83EAE82EF12C25E730E012
:101B50004FE251E065E770E087EF90E0FDD99FED3F
:101B6000E92E95E0F92E02E020EE37E040E050E06B
:101B700068EC70E08CE390E00E94990580912C065F
:101B800090912D06892B09F048C0E09189068E2F8F
:101B900090E08830910508F040C0FC01E25BFF4F07
:101BA0000C94BF44E4EAEE2EE4E0FE2E04C07FE98C
:101BB000E72E74E0F72E02E02FE130E04FEF5FEF09
:101BC00065E070E086E490E026C065E9E62E64E01A
:101BD000F62E18C05BE8E52E54E0F52E13C041E860
:101BE000E42E44E0F42E0EC037E7E32E34E0F32E6B
:101BF00009C02DE6E22E24E0F22E04C093E6E92E81
:101C000094E0F92E02E02FE130E04FEF5FEF65E066
:101C100070E08EE190E00E94990580912C069091F1
:101C20002D06019701F580913506813069F038F075
:101C30008230C9F411E8E12E14E0F12E09C085E9E3
:101C4000E82E84E0F82E04C00BE8E02E04E0F02E2D
:101C500002E02FE130E04FEF5FEF65E070E08EE1F2
:101C600090E00E94990580912C0690912D06029794
:101C700001F580913C06813069F038F08230C9F47A
:101C8000F1E8EF2EF4E0FF2E09C0B5E9EB2EB4E049
:101C9000FB2E04C0ABE8EA2EA4E0FA2E02E02FE10E
:101CA00030E04FEF5FEF65E070E08EE190E00E9482
:101CB000990580912C0690912D06049701F580914D
:101CC0009406813069F038F08230C9F461E8E62E7C
:101CD00064E0F62E09C0E5E9EE2EE4E0FE2E04C035
:101CE0007BE8E72E74E0F72E02E02FE130E04FEFC3
:101CF0005FEF65E070E08EE190E00E9499058091D1
:101D00002C0690912D06059701F58091880681306B
:101D100069F038F08230C9F431E8E32E34E0F32E74
:101D200009C055E9E52E54E0F52E04C04BE8E42E39
:101D300044E0F42E02E02FE130E04FEF5FEF65E08A
:101D400070E08EE190E00E94990580912C069091C0
:101D50002D06069701F580918506813069F038F0EF
:101D60008230C9F481E8E82E84E0F82E09C025E924
:101D7000E22E24E0F22E04C09BE8E92E94E0F92E36
:101D800002E02FE130E04FEF5FEF65E070E08EE1C1
:101D900090E00E9499051F910F91FF90EF90DF90C6
:101DA000CF900895EF92FF920F931F938091230697
:101DB000909124060A97A8F48091FA0581110CC02D
:101DC0000FE110E02CE330E044E650E06BE470E01B
:101DD0008EE690E00E94A40481E08093FA051092C0
:101DE0002E0680912306909124060A978A35910544
:101DF000A8F480912E0681110CC00FE110E02CE3B5
:101E000030E044E650E06BE470E08EE690E00E9443
:101E1000A40481E080932E061092FA058091230697
:101E20009091240684369105A0F080912E06813091
:101E300061F40FE110E02CE330E044E650E06BE4A5
:101E400070E08EE690E00E94A40410922E0610929C
:101E5000FA0580912A0690912B06019779F4E0907B
:101E60002306F090240603E02FE130E04FEF5FEF10
:101E700064E670E082E890E00E94DF0580912A0627
:101E800090912B06892B79F4E0902306F09024069C
:101E900003E02FE130E040E058EF64E670E082E8D4
:101EA00090E00E94DF051F910F91FF90EF90089541
:101EB000EF92FF920F931F938091560690915706D1
:101EC0000A97A8F480912206811111C00FE110E059
:101ED00027E330E048E550E06BE970E088E090E00F
:101EE0000E94A40481E080932206109286068091CD
:101EF00056069091570684369105D8F480912306B2
:101F0000909124060A97A8F080918606811111C04D
:101F10000FE110E027E330E048E550E06BE970E0C6
:101F200088E090E00E94A40481E0809386061092ED
:101F30002206809156069091570684369105A0F0AE
:101F400080918606813061F40FE110E027E330E0F4
:101F500048E550E06BE970E088E090E00E94A4045E
:101F60001092860610922206E0905606F0905706D0
:101F700003E02FE130E04FEF5FEF64EB70E08FE0C4
:101F800090E00E94DF051F910F91FF90EF90089560
:101F9000EF92FF920F931F93809143069091440616
:101FA0000A97A8F48091290681110CC00FE110E076
:101FB00024E230E04AE550E064E670E088E090E03A
:101FC0000E94A40481E0809329061092400680912B
:101FD0004306909144060A978A359105A8F48091AA
:101FE000400681110CC00FE110E024E230E04AE528
:101FF00050E064E670E088E090E00E94A40481E094
:1020000080934006109229068091430690914406E1
:1020100084369105A1F480914006813061F40FE18E
:1020200010E024E230E04AE550E064E670E088E049
:1020300090E00E94A404109229061092400680911C
:102040004306909144068436910530F084E690E092
:102050009093440680934306E0904306F090440634
:1020600003E02FE130E04FEF5FEF6EE670E084E1D8
:1020700090E00E94DF0580919506909196060A9760
:10208000A8F480918F06811111C00FE110E024E2C5
:1020900030E04AE550E064E670E08FED90E00E94A9
:1020A000A40481E080938F061092580680919506D3
:1020B000909196060A978A359105A8F48091580662
:1020C000811111C00FE110E024E230E04AE550E058
:1020D00064E670E08FED90E00E94A40481E08093BC
:1020E000580610928F068091950690919606843638
:1020F000910529F410928F061092580603C0843679
:10210000910530F084E690E09093960680939506D2
:10211000E0909506F090960603E02FE130E04FEF57
:102120005FEF6EE670E089EE90E00E94DF051F91A0
:102130000F91FF90EF900895CF93DF9300D000D0E0
:10214000CDB7DEB7809163001C821B821A82198290
:10215000BE016F5F7F4FCE0103960E9422438B81A9
:102160009C81853C9940A0F0A89589819A81843C06
:10217000994070F4A89589819A818D3D954040F0F1
:10218000A89581E090E090932B0680932A06A8956D
:102190000F900F900F900F90DF91CF910895CF93F4
:1021A000DF9300D000D0CDB7DEB7A8958091630053
:1021B0001C821B821A821982BE016F5F7F4FCE0183
:1021C00003960E9422438B819C81853C9940A8F014
:1021D00089819A81843C994080F489819A818D3DDE
:1021E000954058F010922B0610922A068FE19EE43B
:1021F0000197F1F700C00000A8950F900F900F9085
:102200000F90DF91CF9108957F928F929F92AF921E
:10221000BF92CF92DF92EF92FF920F931F93CF93D3
:10222000DF93EC016B015A014901702EA895809152
:10223000FD059091FE050A97A8F480918A06811108
:1022400011C00FE110E02EE130E044E650E06550AF
:102250007109CE0144970E94A40481E080938A060C
:1022600010924B068091FD059091FE050A978A35E4
:102270009105C0F480914B06811114C00FE110E06C
:102280002EE130E044E650E0B60165507109CE0120
:1022900044970E94A40481E080934B0610928A0622
:1022A000109225068091FD059091FE0584369105DA
:1022B000C0F080912506811114C00FE110E02EE1DD
:1022C00030E044E650E0B60165507109CE01449714
:1022D0000E94A40481E08093250610924B06109280
:1022E0008A06E090FD05F090FE05072D9401A501FA
:1022F000B601CE010E94DF05A895DF91CF911F9115
:102300000F91FF90EF90DF90CF90BF90AF909F9094
:102310008F907F900895CF92DF92EF92FF920F936C
:102320001F938FE190E00E941906A89500EE17E038
:1023300021E430E048EC50E06AEA70E085E090E0AB
:102340000E94A4040FEF1FEF21E430E048EC50E0BE
:1023500063E270E085E090E00E94000789E4E82EE7
:1023600082E0F82E01E02FE130E040EE57E06CE330
:1023700070E088E290E00E9499050FEF1FEF20E5E2
:1023800030E040E550E065E070E08BEE90E00E94C8
:10239000000790EEC92E97E0D92E24E1E22EF12C11
:1023A00003E111E026E430E041E351E066E470E04F
:1023B00085EF90E00E94AC0737E1E32EF12C24E496
:1023C00030E04FE251E064E470E087EF90E00E947B
:1023D000AC070FEF1FEF20E530E040E550E064E68A
:1023E00070E08BEE90E00E94000745EAE42EF12CAD
:1023F00003E111E023E730E041E351E063E770E0FF
:1024000085EF90E00E94AC0753EAE52EF12C25E71A
:1024100030E04FE251E065E770E087EF90E00E9426
:10242000AC0766E4E62E65E0F62E02E020EE37E02B
:1024300040E050E068EC70E08DE290E00E94990589
:102440008FE19EE40197F1F700C000001F910F910A
:10245000FF90EF90DF90CF900895A8958091480667
:10246000813071F4A49A80E185BBA8952FEF82E5B5
:1024700097E0215080409040E1F700C0000015BA7D
:10248000A8950895A89580914806813021F5A49AD1
:1024900080E185BB2FEF32E597E02150304090403E
:1024A000E1F700C00000A89515BA2FEF32E597E0DC
:1024B000215030409040E1F700C00000A89585BB56
:1024C0002FEF32E587E0215030408040E1F700C037
:1024D0000000A89515BA0895A89580914806813006
:1024E00009F048C0A49A80E185BBA8952FEF32E59A
:1024F00097E0215030409040E1F700C00000A895DF
:1025000015BAA8952FEF32E597E021503040904062
:10251000E1F700C00000A89585BBA8952FEF32E534
:1025200097E0215030409040E1F700C00000A895AE
:1025300015BAA8952FEF32E597E021503040904032
:10254000E1F700C00000A89585BB2FEF32E587E0DA
:10255000215030408040E1F700C00000A89515BA36
:102560009FEF22E537E0915020403040E1F700C076
:102570000000A8950895A895109245061092390676
:102580001092F80510925B061092360610922806FB
:102590001092470610923F06109255061092F905C8
:1025A00083EB92E00E94DA4780934806A89584EB7B
:1025B00092E00E94E24790933B0680933A06A895EA
:1025C00080912C0690912D06892B51F5A895E091CC
:1025D00089068E2F90E08830910510F5FC01EA5AAB
:1025E000FF4F4EE150E00C94BF4464E972E014C028
:1025F00066E772E011C068E572E00EC06AE372E05F
:102600000BC06CE172E008C06EEF71E005C060EED7
:1026100071E002C062EC71E083E096E00E94CA477C
:10262000A89580912C0690912D060197D1F4A8953C
:1026300080913506813069F038F0823091F44EE1B6
:1026400050E068E671E009C04EE150E064EA71E0F4
:1026500004C04EE150E066E871E083E096E00E943D
:10266000CA47A89580912C0690912D060297D1F427
:10267000A89580913C06813069F038F0823091F461
:102680004EE150E06EE071E009C04EE150E06AE4D6
:1026900071E004C04EE150E06CE271E083E096E04E
:1026A0000E94CA47A89580912C0690912D06049708
:1026B000C9F480919406813069F038F0823091F449
:1026C0004EE150E064EB70E009C04EE150E060EF95
:1026D00070E004C04EE150E062ED70E083E096E00F
:1026E0000E94CA47A89580912C0690912D060597C7
:1026F000C9F480918806813069F038F0823091F415
:102700004EE150E06AE570E009C04EE150E066E954
:1027100070E004C04EE150E068E770E083E096E0CE
:102720000E94CA47A89580912C0690912D06069785
:10273000C9F480918506813069F038F0823091F4D7
:102740004EE150E060E070E009C04EE150E06CE323
:1027500070E004C04EE150E06EE170E083E096E08E
:102760000E94CA47A89587EC90E00197F1F700C056
:10277000000080910306909104069093F7058093E2
:10278000F605809105069091060690934A0680937F
:1027900049068091070690910806909392068093CF
:1027A00091068091090690910A06909334068093D1
:1027B000330680910B0680935E0680910D06909102
:1027C0000E06909332068093310680910F06809317
:1027D00042068091110680934106809113068093F2
:1027E000F2058091150690911606909382068093CB
:1027F0008106809117069091180690935D0680934C
:102800005C0680912C0690912D06079741F48091EB
:10281000190690911A0690932D0680932C068091AC
:102820001B0690911C069093800680937F068091F2
:102830001D0690911E0690930206809301068091DA
:102840001F06909120069093270680932606A89550
:1028500008951092960610929506BC9A809195065E
:10286000880F81BF1092440610924306139A8091FC
:102870004306880F809386002FDE8DE490E09093CE
:102880008C0680938B0681E090E090932B068093DA
:102890002A060895CF934091FD055091FE052091A1
:1028A000330630913406429FC001439F900D529FE2
:1028B000900D11246AE070E00E94AB4470935A06B8
:1028C00060935906809143069091440685369105A0
:1028D00030F084E690E09093440680934306809124
:1028E000410690E0209143063091440682179307F9
:1028F00020F49093440680934306209145062111CD
:1029000014C020915606309157062233310538F411
:1029100024E630E0309344062093430606C0223379
:10292000310519F021E0209345062091450640919C
:10293000490650914A062130E1F520914306309135
:1029400044062436310530F024E630E03093440666
:10295000209343066417750760F5E0915606F091E1
:1029600057062091430630914406E617F707C0F456
:102970002F5F3F4F8217930728F030934406209330
:10298000430604C090934406809343062091430677
:10299000309144062536310560F024E630E005C06C
:1029A0002115310531F0215031093093440620932F
:1029B00043064617570708F04AC020915606309143
:1029C000570624173507D0F46091430670914406EA
:1029D0006F5F7F4F6536710510F064E670E07093AD
:1029E000440660934306609143067091440686173F
:1029F000970720F4909344068093430642175307A9
:102A000030F58091430690914406009729F0019794
:102A10009093440680934306241B350B2B303105DD
:102A2000B0F080914306909144060A9720F41092EA
:102A300044061092430680914306909144068A30E2
:102A4000910528F00A979093440680934306C0911D
:102A50005E06C130D1F480913906811116C02091F3
:102A60002306309124068091310690913206281772
:102A7000390759F4809156069091570690934A066B
:102A800080934906EADCC0933906C091F205C13053
:102A900009F58091F80581111DC080912306909160
:102AA00024062091810630918206821B930B0597A4
:102AB00088F42091490630914A0680915C069091F5
:102AC0005D06820F931F90934A0680934906C5DCEA
:102AD000C093F805CF91089580915B0681111CC0C9
:102AE0008091230690912406209131063091320680
:102AF000821B930B029780F482E390E090939606FA
:102B00008093950681E080935B06809328068091F0
:102B10005E06811101C0A1DC2091310630913206A0
:102B200060918D0670918E064091910650919206AB
:102B3000649FC001659F900D749F900D11246AE001
:102B400070E00E94AB44620F731F7093F5056093B1
:102B5000F405E0919506F09196064091F6055091A6
:102B6000F7054617570720F45093F5054093F405F1
:102B70008091420690E08E179F0720F4909396066E
:102B80008093950680912306909124062817390793
:102B900020F048175907A0F176C020915506211161
:102BA000F8CF84179507A8F76091F4057091F505A3
:102BB00020919506309196068617970788F42F5F27
:102BC0003F4F2536310528F430939606209395061D
:102BD000E0CF24E630E03093960620939506A6C019
:102BE0002115310531F0215031093093960620939B
:102BF00095062091950630919606232B51F296C0AA
:102C000020919506309196062115310531F021501D
:102C100031093093960620939506841B950B0697F1
:102C2000B0F080919506909196060A9720F4109244
:102C300096061092950680919506909196068A3098
:102C4000910528F00A9790939606809395068091B7
:102C5000F905811106C016DC81E080933F06809360
:102C6000F9052091FF053091000680913A06909178
:102C70003B068217930738F4ECDD81E090E09093F7
:102C80002B0680932A0680913606811158C0409108
:102C90007F0650918006809131069091320684170C
:102CA000950708F04CC0E0912306F09124064E17DA
:102CB0005F0729F481E08093550680934706809151
:102CC00055068130E1F56091FB057091FC0520917E
:102CD00001063091020662177307A8F480919506E9
:102CE00090919606E417F50738F40196853691051C
:102CF00030F084E690E003C0009729F001979093AC
:102D000096068093950626173707C8F41092550645
:102D100080918D0690918E06821B930B90938E0668
:102D200080938D0681E080933606089548175907F1
:102D300008F0A9CF209195063091960668CF0895A6
:102D400080915B0681111BC02091230630912406DF
:102D500080913106909132068217930780F482E3C6
:102D600090E0909396068093950681E080935B06B1
:102D70008093280680915E06811101C06EDBE09190
:102D80003106F091320640918D0650918E062091C9
:102D9000910630919206429FC001439F900D529F31
:102DA000900D11246AE070E00E94AB446E0F7F1F0B
:102DB0007093F5056093F405209195063091960681
:102DC0004091F6055091F7054617570720F45093A8
:102DD000F5054093F4058091420690E08217930731
:102DE00020F49093960680939506209123063091C7
:102DF0002406E217F30700F58091550681111CC0E7
:102E000024173507C8F46091F4057091F505809199
:102E10009506909196062617370738F40196853661
:102E2000910530F084E690E003C0009729F0019707
:102E3000909396068093950642175307E0F580918C
:102E40009506909196060197909396068093950625
:102E5000241B350B2630310590F00A9720F4109290
:102E600096061092950680919506909196068A3066
:102E7000910528F00A979093960680939506809185
:102E8000F905811106C0FEDA81E080933F06809348
:102E9000F9052091FF053091000680913A06909146
:102EA0003B068217930738F4D4DC81E090E09093DE
:102EB0002B0680932A068091360681114EC04091E0
:102EC0007F065091800680913106909132068417DA
:102ED000950708F042C0E0912306F09124064E17B2
:102EE0005F0729F481E0809355068093470680911F
:102EF0005506813091F56091FB057091FC0520919C
:102F000001063091020662177307A8F480919506B6
:102F100090919606E417F50738F4019685369105E9
:102F200030F084E690E003C0009729F00197909379
:102F30009606809395062617370778F41092550663
:102F400080918D0690918E06821B930B90938E0636
:102F500080938D0681E0809336060895CF93C091CB
:102F60005E06C130D1F480913906811116C02091DE
:102F7000230630912406809131069091320628175D
:102F8000390759F4809156069091570690934A0656
:102F90008093490662DAC09339064091FD0550914D
:102FA000FE052091330630913406429FC001439FB5
:102FB000900D529F900D11246AE070E00E94AB4486
:102FC00070935A0660935906809143069091440687
:102FD0008536910530F084E690E090934406809326
:102FE00043068091410690E02091430630914406CB
:102FF0008217930720F49093440680934306209110
:103000004506211114C020915606309157062639E5
:10301000310538F424E630E030934406209343062B
:1030200006C02639310519F021E02093450620918C
:1030300045064091490650914A06213079F56417BA
:10304000750760F5E0915606F0915706209143060A
:1030500030914406E617F707C0F42F5F3F4F821701
:10306000930728F0309344062093430604C09093BE
:10307000440680934306209143063091440625364A
:10308000310560F024E630E005C02115310531F04E
:1030900021503109309344062093430646175707C1
:1030A00008F088C020915E06211133C02091560699
:1030B0003091570624173507D0F46091430670917C
:1030C00044066F5F7F4F6536710510F064E670E06F
:1030D00070934406609343066091430670914406E2
:1030E0008617970720F4909344068093430642176F
:1030F000530708F05FC08091430690914406009703
:1031000029F001979093440680934306241B350BC6
:1031100038C0213009F04EC020912306309124069A
:10312000609131067091320626173707D0F440912E
:103130004306509144064F5F5F4F4536510510F0EE
:1031400044E650E0509344064093430640914306C2
:10315000509144068417950720F490934406809379
:1031600043066217730730F5809143069091440639
:10317000009729F001979093440680934306261BFD
:10318000370B2B303105B0F0809143069091440607
:103190000A9720F410924406109243068091430649
:1031A000909144068A30910528F00A97909344063E
:1031B00080934306CF9108954091FD055091FE05FF
:1031C0002091330630913406429FC001439F900DF9
:1031D000529F900D11246AE070E00E94AB447093FE
:1031E0005A066093590680914306909144068536AD
:1031F000910530F084E690E0909344068093430676
:103200008091410690E02091430630914406821758
:10321000930720F49093440680934306209145063B
:103220004091560650915706211110C0463951055C
:1032300038F424E630E0309344062093430606C079
:103240004639510519F021E02093450620914506A5
:10325000E0914906F0914A06213059F56E177F0733
:1032600040F5209143063091440646175707C0F4B5
:103270002F5F3F4F8217930728F030934406209327
:10328000430604C09093440680934306209143066E
:10329000309144062536310560F024E630E005C063
:1032A0002115310531F02150310930934406209326
:1032B0004306E617F70708F046C04E175F07D0F43D
:1032C00020914306309144062F5F3F4F253631054C
:1032D00010F024E630E0309344062093430620911A
:1032E0004306309144068217930720F490934406D6
:1032F00080934306E417F50730F5809143069091DB
:103300004406009729F00197909344068093430662
:10331000CA018E1B9F0B0B97B0F0809143069091D2
:1033200044060A9720F410924406109243068091B6
:103330004306909144068A30910528F00A979093AD
:103340004406809343068091420690E020919506C2
:10335000309196068217930720F4909396068093F7
:103360009506E417F50770F48091950690919606FE
:1033700001968536910510F084E690E090939606CC
:103380008093950608954091FD055091FE0520918A
:10339000330630913406429FC001439F900D529FE7
:1033A000900D11246AE070E00E94AB4470935A06BD
:1033B00060935906809143069091440685369105A5
:1033C00030F084E690E09093440680934306809129
:1033D000410690E0209143063091440682179307FE
:1033E00020F49093440680934306209145062111D2
:1033F00014C020915606309157062639310538F40D
:1034000024E630E0309344062093430606C0263974
:10341000310519F021E020934506209145064091A1
:10342000490650914A06213079F56417750760F511
:10343000E0915606F09157062091430630914406DC
:10344000E617F707C0F42F5F3F4F8217930728F066
:10345000309344062093430604C09093440680931F
:10346000430620914306309144062536310560F02D
:1034700024E630E005C02115310531F02150310935
:1034800030934406209343064617570708F04AC076
:10349000209156063091570624173507D0F46091D5
:1034A0004306709144066F5F7F4F6536710510F0DB
:1034B00064E670E0709344066093430660914306AF
:1034C000709144068617970720F4909344068093E2
:1034D00043064217530730F5809143069091440606
:1034E000009729F001979093440680934306241B8C
:1034F000350B2B303105B0F0809143069091440696
:103500000A9720F4109244061092430680914306D5
:10351000909144068A30910528F00A9790934406CA
:10352000809343060895BC9A80919506880F81BFC9
:10353000139A80914306880F8093860080912C0611
:1035400090912D06892B11F4A5D9C6DA80912C060D
:1035500090912D06019729F410924406109243068B
:10356000EFDB80912C0690912D06029729F41092A2
:10357000960610929506F2DC80912C0690912D060D
:10358000049709F419DE80912C0690912D06059779
:1035900009F412DE80912C0690912D06069709F40D
:1035A000F2CE089563EC70E084E992E00E94FD475A
:1035B00062EC71E086E992E00E94FD4766E170E00E
:1035C00088E992E00E94FD4766E170E08AE992E0B6
:1035D0000E94FD4761E070E08CE992E00E94FD47A7
:1035E000A8956EE670E08EE992E00E94FD4764E6E1
:1035F00070E080EA92E00E94FD4764E670E082EAB3
:1036000092E00E94FD4760E070E084EA92E00E9450
:10361000FD47A89560E070E086EA92E00E94FD47D1
:1036200060E070E088EA92E00E94FD4760E070E0B0
:103630008AEA92E00E94FD4760E070E08CEA92E046
:103640000E94FD4760E070E08EEA92E00E94FD4734
:1036500060E070E080EB92E00E94FD47A89566EE86
:1036600070E086E792E00E94FD4762EC71E088E737
:1036700092E00E94FD4766E170E08AE792E00E94D6
:10368000FD4766E170E08CE792E00E94FD4761E053
:1036900070E08EE792E00E94FD47A89563E770E036
:1036A00080E892E00E94FD4764E670E082E892E0E4
:1036B0000E94FD4764E670E084E892E00E94FD47C6
:1036C00060E070E086E892E00E94FD4760E070E014
:1036D00088E892E00E94FD4760E070E08AE892E0AE
:1036E0000E94FD47A89560E070E08CE892E00E949F
:1036F000FD4760E070E08EE892E00E94FD4760E0E8
:1037000070E080E992E00E94FD4760E070E082E9AD
:1037100092E00E94FD47A89566EE70E088E592E091
:103720000E94FD4762EC71E08AE592E00E94FD474D
:1037300066E170E08CE592E00E94FD4766E170E092
:103740008EE592E00E94FD4761E070E080E692E045
:103750000E94FD47A89563E770E082E692E00E9430
:10376000FD4764E670E084E692E00E94FD4764E66F
:1037700070E086E692E00E94FD4760E070E088E637
:1037800092E00E94FD4760E070E08AE692E00E94CD
:10379000FD4760E070E08CE692E00E94FD47A8954E
:1037A00060E070E08EE692E00E94FD4760E070E02D
:1037B00080E792E00E94FD4760E070E082E792E0DF
:1037C0000E94FD4760E070E084E792E00E94FD47C0
:1037D000A89566E970E08AE392E00E94FD4768ECF4
:1037E00070E08CE392E00E94FD4766E170E08EE3BA
:1037F00092E00E94FD4766E170E080E492E00E9462
:10380000FD4761E070E082E492E00E94FD47A895E8
:1038100063E770E084E492E00E94FD4764E670E0B4
:1038200086E492E00E94FD4764E670E088E492E05E
:103830000E94FD4760E070E08AE492E00E94FD474C
:1038400060E070E08CE492E00E94FD4760E070E090
:103850008EE492E00E94FD47A89560E070E080E56C
:1038600092E00E94FD4760E070E082E592E00E94F5
:10387000FD4760E070E084E592E00E94FD4760E073
:1038800070E086E592E00E94FD47A8956EEB70E03F
:103890008CE192E00E94FD4768EC70E08EE192E0DE
:1038A0000E94FD4766E170E080E292E00E94FD47E1
:1038B00066E170E082E292E00E94FD4761E070E024
:1038C00084E292E00E94FD47A89564E670E086E2FB
:1038D00092E00E94FD4764E670E088E292E00E9478
:1038E000FD4764E670E08AE292E00E94FD4760E0F6
:1038F00070E08CE292E00E94FD4760E070E08EE2B2
:1039000092E00E94FD4760E070E080E392E00E9458
:10391000FD47A89560E070E082E392E00E94FD47D9
:1039200060E070E084E392E00E94FD4760E070E0B8
:1039300086E392E00E94FD4760E070E088E392E059
:103940000E94FD47A89566EE70E08EEF91E00E9420
:10395000FD4762EC71E080E092E00E94FD4766E185
:1039600070E082E092E00E94FD4766E170E084E052
:1039700092E00E94FD4761E070E086E092E00E94E4
:10398000FD47A89563E770E088E092E00E94FD475C
:1039900064E670E08AE092E00E94FD4764E670E031
:1039A0008CE092E00E94FD4760E070E08EE092E0E3
:1039B0000E94FD4760E070E080E192E00E94FD47D8
:1039C00060E070E082E192E00E94FD47A89560E02F
:1039D00070E084E192E00E94FD4760E070E086E1E3
:1039E00092E00E94FD4760E070E088E192E00E9472
:1039F000FD4760E070E08AE192E00E94FD47A895F3
:103A000066EE70E080EE91E00E94FD4762EC71E0AE
:103A100082EE91E00E94FD4766E170E084EE91E065
:103A20000E94FD4766E170E086EE91E00E94FD474E
:103A300061E070E088EE91E00E94FD47A89563E7A1
:103A400070E08AEE91E00E94FD4764E670E08CEE43
:103A500091E00E94FD4764E670E08EEE91E00E94E6
:103A6000FD4760E070E080EF91E00E94FD4760E07C
:103A700070E082EF91E00E94FD4760E070E084EF2B
:103A800091E00E94FD47A89560E070E086EF91E02C
:103A90000E94FD4760E070E088EF91E00E94FD47E2
:103AA00060E070E08AEF91E00E94FD4760E070E026
:103AB0008CEF91E00E94FD47A89563EC70E084EAEA
:103AC00091E00E94FD4766E170E088EA91E00E9483
:103AD000FD4761E070E08CEA91E00E94FD476FE0F5
:103AE00070E08EEA91E00E94FD47A89564E670E0E0
:103AF00080EB91E00E94FD4761E070E08AEB91E08D
:103B00000E94FD4763EC70E08CEB91E00E94FD4762
:103B10006AE070E08EEB91E00E94FD47A89562ECB0
:103B200071E08CE491E00E94FD4766E170E080E581
:103B300091E00E94FD4761E070E082E591E00E9423
:103B4000FD476EE670E084E591E00E94FD47A89590
:103B500064E670E088E591E00E94FD4762E070E075
:103B600080E691E00E94FD4762EC71E082EF90E018
:103B70000E94FD4766E170E084EF90E00E94FD47FF
:103B800062E170E086EF90E00E94FD47A89564E650
:103B900070E08CEF90E00E94FD4764E670E08EEFED
:103BA00090E00E94FD4764E070E086E091E00E94B2
:103BB000FD476CE271E08CE091E00E94FD47A89522
:103BC00062EC71E088E990E00E94FD4766E170E0F8
:103BD0008AE990E00E94FD4766E170E08CE990E0A0
:103BE0000E94FD4761E070E08EE990E00E94FD4791
:103BF000A8956EE670E080EA90E00E94FD4764E6DA
:103C000070E082EA90E00E94FD4764E670E084EA9A
:103C100090E00E94FD4765E070E08CEA90E00E9431
:103C2000FD47A89562EC71E08EE390E00E94FD47AD
:103C300066E170E082E490E00E94FD4761E070E0A0
:103C400084E490E00E94FD476EE670E086E490E038
:103C50000E94FD47A89564E670E08AE490E00E9427
:103C6000FD4766E070E082E590E00E94FD4763EC6E
:103C700070E084E992E00E94FD47A89508956FE006
:103C800070E088EB92E00E94FD476FE070E086EB09
:103C900092E00E94FD476FE070E084EB92E00E94AA
:103CA000FD4761E083EB92E00E94F04761E082EB28
:103CB00092E00C94F0478FB9779BFECF8FB10895B7
:103CC000CF93A39AAB9AAB9880E0F5DFC82F80E042
:103CD000F2DFAB9A6C2F70E0762F6627682B687F37
:103CE0007F7723E0769567952A95E1F780E090E06D
:103CF0000E94BA4320E030E040E85EE30E942044A6
:103D00000E948E437093240660932306CB01CF91CB
:103D10000895CF93A79AAF9AAF9880E0CCDFC82FD1
:103D200080E0C9DFAF9A6C2F70E0762F6627682B92
:103D3000687F7F7723E0769567952A95E1F780E0A5
:103D400090E00E94BA4320E030E040E85EE30E9449
:103D500020440E948E437093570660935606CB0111
:103D6000CF91089580E091E090939F0680939E0606
:103D7000809124068F93809123068F938EE091E0AB
:103D80009F938F930E94FA448DE08A95F1F700008B
:103D90008091FE058F938091FD058F9388E191E0DE
:103DA0009F938F930E94FA449DE09A95F1F700004B
:103DB000809144068F93809143068F9382E291E035
:103DC0009F938F930E94FA448DE08A95F1F700004B
:103DD000809196068F93809195068F938DE291E066
:103DE0009F938F930E94FA449DE09A95F1F700000B
:103DF00087E391E09F938F930E94FA448DE08A9528
:103E0000F1F70000809157068F93809156068F93AB
:103E10008FE391E09F938F930E94FA44A8958DB70A
:103E20009EB746960FB6F8949EBF0FBE8DBF809189
:103E30002A0690912B06892B41F488E491E09F9308
:103E40008F930E94FA440F900F90A89580912A06B4
:103E500090912B06019741F48FE491E09F938F930B
:103E60000E94FA440F900F909DE09A95F1F70000A0
:103E7000E0912C06F0912D06E830F10508F09CC089
:103E8000E25AFF4F0C94BF4486E591E09F938F93D5
:103E90000E94FA44A8950F900F90E09189068E2F0A
:103EA00090E08830910508F087C0FC01EA59FF4F87
:103EB0000C94BF4485E691E071C085E791E06EC047
:103EC0008DEA91E06BC08CEB91E068C08BEC91E0E7
:103ED00065C08AED91E09F938F930E94FA44A89564
:103EE0000F900F9080913506813009F452C008F48C
:103EF0004DC0823009F450C008958AEE91E09F933E
:103F00008F930E94FA44A8950F900F9080913C06E1
:103F1000813009F43EC0D0F1823009F43DC00895EB
:103F20008BEF91E042C089E092E09F938F930E94D3
:103F3000FA44A8950F900F9080919406813049F132
:103F400028F1823049F108958AE192E09F938F939E
:103F50000E94FA44A8950F900F90809188068130B6
:103F6000C1F0A0F08230C1F008958DE292E09F93FD
:103F70008F930E94FA44A8950F900F908091850628
:103F8000813039F018F0823039F0089580E891E0FE
:103F900005C08FE891E002C08EE991E09F938F9376
:103FA0000E94FA4407C08FE392E09F938F930E9490
:103FB000FA44A8950F900F900895CF92DF92EF9258
:103FC000FF920F931F93CF93DF9300D000D0CDB714
:103FD000DEB780912A0690912B06019709F045C122
:103FE00080913D0690913E06892BD9F40FE110E0B7
:103FF00024E230E04AE550E064E670E088E090E0DA
:104000000E94A40424E230E04AE550E064E670E057
:104010008FED90E00E94A404A895A49AAC980E9409
:10402000EB07CC24C394D12C80912A0690912B06C7
:10403000019709F01AC1A89595DE80918B069091A1
:104040008C068A35910549F42FEF8DE399E42150D0
:1040500080409040E1F700C00000A89503E02FE108
:1040600030E04FEF5FEF69E170E085E890E00E949B
:10407000041180916300A8951C821B821A82198208
:10408000BE016F5F7F4FCE0103960E9422438B815A
:104090009C818431954088F489819A81883D9E4035
:1040A00060F489819A81853C994038F0D0923E062F
:1040B000C0923D0610924D0626D48B819C8184319E
:1040C000954008F03FC089819A818C3D9540D0F59C
:1040D00089819A81853F9140A8F1D0923E06C09295
:1040E0003D0610925F0680912C0690912D06892B3B
:1040F00011F40E94233380912C0690912D06019794
:1041000011F40E94BF3B80912C0690912D060297DE
:1041100011F40E94C63C80912C0690912D060497C4
:1041200011F40E94CD3D80912C0690912D060597AB
:1041300009F471D580912C0690912D06069711F403
:104140000E941B328091F105813019F58B819C8191
:10415000853C9940F0F089819A818C3D9540C8F466
:1041600089819A81853F9140A0F0D0923E06C0920D
:104170003D060E948B1180E00E94E4410E944E4265
:1041800010923E0610923D068FE190E00E941906C3
:1041900014DF96DD0E94D20EA8958FEF91EE24E0F9
:1041A000815090402040E1F700C00000B2DDA895AA
:1041B0000E94580FE0904306F090440603E02FE180
:1041C00030E04FEF5FEF6EE670E08CE190E00E9430
:1041D000DF05E0909506F09096062FE130E04FEF76
:1041E0005FEF6EE670E080EF90E00E94DF05809167
:1041F000F105813011F40E94D6420E94CF108091C7
:104200002A0690912B06892B09F00ECFA8950E94C3
:10421000BB12A8950E942D120E94EB070FE110E03F
:1042200024E230E04AE550E064E670E088E090E0A7
:104230000E94A40424E230E04AE550E064E670E025
:104240008FED90E00E94A4048091F105813021F46B
:104250000E94DF410E94F2421092FE051092FD057D
:1042600010923E0610923D06DFCE0F900F900F90F9
:104270000F90DF91CF911F910F91FF90EF90DF9002
:10428000CF900895EF92FF920F931F93CF93809159
:104290004C06813009F04BC18FE190E00E94190675
:1042A0000E94C10B85E080935206C5E080914C06C8
:1042B000813009F03CC10E94DD0C809152068230B1
:1042C000D9F480917E068F5F80937E060FE110E027
:1042D0002CE330E046EE50E069E670E081E090E0EB
:1042E0000E94A40422E330E043EC50E068E270E076
:1042F00088E090E00E94A404809152068330D9F4B3
:1043000080917E06815080937E060FE110E02CE3C1
:1043100030E046EE50E069E670E081E090E00E9417
:10432000A40422E330E043EC50E068E270E088E06F
:1043300090E00E94A40480917E06853010F01092D7
:104340007E0680917E06823081F1B8F48823D9F010
:10435000813009F0C1C076E9E72E75E0F72E01E063
:104360002FE130E04FEF5FEF6CE370E088E090E02A
:104370000E94990586EB92E029C08330B1F1843028
:1043800009F471C0A9C0EFEAEE2EE5E0FE2E01E0CF
:104390002FE130E04FEF5FEF6CE370E08FE090E0F3
:1043A0000E94990588EB92E011C06AE8E62E65E06C
:1043B000F62E01E02FE130E04FEF5FEF6CE370E0AD
:1043C00082E390E00E94990584EB92E00E94E2472C
:1043D0007C0103E02FE130E04FEF5FEF62E870E037
:1043E00080E590E00E94DF0577C042E7E42E45E0DB
:1043F000F42E01E02FE130E04FEF5FEF6CE370E06F
:1044000088E290E00E94990550E8E52E55E0F52EEF
:1044100002E02FE130E04FEF5FEF62E870E088E20A
:1044200090E00E94990580915206811119C0BAD876
:1044300026DC3CE3E32E35E0F32E2FE130E04FEFB6
:104440005FEF62E870E088E290E00E9499052FEF4C
:1044500089E698E1215080409040E1F700C00000DB
:10446000C093520639C021E6E22E25E0F22E01E08B
:104470002FE130E04FEF5FEF6CE370E08EE190E012
:104480000E94990583EB92E00E94DA47813079F42B
:1044900093E5E92E95E0F92E03E02FE130E04FEFB0
:1044A0005FEF62E870E080E590E00E94990583EBA1
:1044B00092E00E94DA4781110FC08EE4E82E85E079
:1044C000F82E03E02FE130E04FEF5FEF62E870E09D
:1044D00080E590E00E94990580915206813089F430
:1044E00010924C0610923E0610923D068FE190E02D
:1044F0000E94190681E090E090932B0680932A0693
:104500005CDD80915206811106C081E080934C06EB
:104510001092900612D0C09352062FE785EB91E0DF
:10452000215080409040E1F700C00000BFCECF9105
:104530001F910F91FF90EF900895BF92CF92DF925D
:10454000EF92FF920F931F93CF93DF93809190068A
:104550008111CFC185E080935206C9E1D0E025E00A
:10456000C22ED12C35E0B32E809190068111C1C1AD
:1045700080917E06813009F46FC038F0823009F4F2
:10458000DDC0843009F441C1A4C188EB92E00E94EF
:10459000E2477C0103E02FE130E040E058EF62E8C1
:1045A00070E080E590E00E94DF0588EB92E00E94D9
:1045B000E24790935106809350060E94DD0C809153
:1045C00052068230A9F480915006909151060196CE
:1045D00090935106809350060FE110E02CE330E0F9
:1045E00046EE50E069E670E081E090E00E94A404AD
:1045F000809152068330A9F4809150069091510623
:10460000019790935106809350060FE110E02CE340
:1046100030E046EE50E069E670E081E090E00E9414
:10462000A40480915006909151064A9720F0D093AF
:104630005106C093500680915006909151060A97FA
:1046400020F4D0935106C0935006609150067091AB
:10465000510688EB92E066C086EB92E00E94E2474A
:104660007C0103E02FE130E040E058EF62E870E0C9
:1046700080E590E00E94DF0586EB92E00E94E24731
:104680009093300680932F060E94DD0C8091520695
:104690008230A9F480912F06909130060196909374
:1046A000300680932F060FE110E02CE330E046EE59
:1046B00050E069E670E081E090E00E94A4048091FF
:1046C00052068330A9F480912F069091300601970D
:1046D0009093300680932F060FE110E02CE330E03A
:1046E00046EE50E069E670E081E090E00E94A404AC
:1046F00080912F06909130064A9720F0D093300693
:10470000C0932F0680912F06909130060A9720F4CF
:10471000D0933006C0932F0660912F06709130061B
:1047200086EB92E00E94FD472FE788E391E021505D
:1047300080409040E1F700C00000CBC084EB92E0E5
:104740000E94E2477C0103E02FE130E040E058EFB7
:1047500062E870E080E590E00E94DF0584EB92E083
:104760000E94E24790934F0680934E060E94DD0C14
:10477000809152068230A9F480914E0690914F06A6
:10478000019690934F0680934E060FE110E02CE3C4
:1047900030E046EE50E069E670E081E090E00E9493
:1047A000A404809152068330A9F480914E06909122
:1047B0004F06019790934F0680934E060FE110E04D
:1047C0002CE330E046EE50E069E670E081E090E0F6
:1047D0000E94A40480914E0690914F064F9720F0BE
:1047E000D0924F06C0924E0680914E0690914F0691
:1047F000059720F4D0924F06C0924E0660914E0667
:1048000070914F0684EB92E08DCF83EB92E00E9493
:10481000DA478093F3050E94DD0C809152068230C6
:1048200089F48091F3058F5F8093F3050FE110E029
:104830002CE330E046EE50E069E670E081E090E085
:104840000E94A40480915206833089F48091F3057C
:1048500081508093F3050FE110E02CE330E046EE49
:1048600050E069E670E081E090E00E94A40480914D
:10487000F305823010F01092F3058091F30581303A
:1048800079F493E5E92E95E0F92E03E02FE130E08D
:1048900040E058EF62E870E080E590E00E94990502
:1048A0008091F30581110FC08EE4E82E85E0F82E8B
:1048B00003E02FE130E040E058EF62E870E080E58F
:1048C00090E00E9499056091F30583EB92E00E94CD
:1048D000F04780915206813049F48093900680938E
:1048E0004C068FE190E00E941906CCDCB092520693
:1048F0003BCEDF91CF911F910F91FF90EF90DF9012
:10490000CF90BF9008954F925F926F927F928F9257
:104910009F92AF92BF92CF92DF92EF92FF920F934E
:104920001F93CF93DF9380914D06811163C18FE177
:1049300090E00E9419060E94330B85E08093520696
:1049400010924C061092460655245394C7E0D0E0CE
:10495000A6E0CA2ED12CB5E0AB2EB12C14E0812EEE
:10496000912C03E0602E712C85E0482E80914D063D
:10497000811140C10E94DD0C80915206823089F481
:10498000809146068F5F809346060FE110E02CE38E
:1049900030E046EE50E069E670E081E090E00E9491
:1049A000A40480915206833089F480914606815098
:1049B000809346060FE110E02CE330E046EE50E035
:1049C00069E670E081E090E00E94A40480914606D0
:1049D000893010F010924606E09146068E2F90E046
:1049E0008930910508F0D4C0FC01E259FF4F0C94C6
:1049F000BF44FEE1EF2EF5E0FF2E02E02FE130E0B4
:104A00004FEF5FEF62E870E088E090E00E94990568
:104A100010924C0610922D0610922C06B9C0E0E1BF
:104A2000EE2EE5E0FE2E02E02FE130E04FEF5FEFEB
:104A300068E770E088E090E00E94990510924C06CB
:104A400081E090E013C072E0E72E75E0F72E02E0FF
:104A50002FE130E04FEF5FEF68E770E088E090E033
:104A60000E94990510924C0682E090E090932D06EA
:104A700080932C068DC066EFE62E64E0F62E02E0F1
:104A80002FE130E04FEF5FEF68E770E088E090E003
:104A90000E94990510924C0670922D0660922C0689
:104AA00077C054EEE52E54E0F52E02E02FE130E021
:104AB0004FEF5FEF68E770E088E090E00E949905B3
:104AC00010924C0690922D0680922C0661C03EED0D
:104AD000E32E34E0F32E02E02FE130E04FEF5FEF02
:104AE0006EE670E088E290E00E94990544EDE42EC5
:104AF00044E0F42E2FE130E04FEF5FEF67E870E025
:104B00008FE090E00E94990510924C06B0922D061D
:104B1000A0922C063DC027ECE22E24E0F22E02E00B
:104B20002FE130E04FEF5FEF68E770E088E090E062
:104B30000E94990510924C06D0922D06C0922C0628
:104B400027C099EAE92E94E0F92E02E02FE130E047
:104B50004FEF5FEF68E770E088E090E00E94990512
:104B600010924C06D0932D06C0932C0611C083EBF7
:104B7000E82E84E0F82E02E02FE130E04FEF5FEF07
:104B800068E770E082E090E00E94990550924C0640
:104B900080915206813011F580914C06813059F494
:104BA00010922D0610922C0610924D068FE190E087
:104BB0000E94190667DB50924D0610923E06109235
:104BC0003D0680912C0690912D0690931A068093B5
:104BD00019068FE190E00E941906EFD94092520623
:104BE0002FEF80E792E0215080409040E1F700C035
:104BF0000000BCCEDF91CF911F910F91FF90EF90FD
:104C0000DF90CF90BF90AF909F908F907F906F90EC
:104C10005F904F900895EF92FF920F931F93CF9361
:104C2000DF93A89580915F068111F4C08FE190E039
:104C30000E9419060E944F0C8091880690E0909384
:104C400038068093370685E080935206C1E0D5E0B0
:104C500080915F068111DEC0A8950E94DD0C8091D5
:104C600052068230A9F48091370690913806019659
:104C700090933806809337060FE110E02CE330E084
:104C800046EE50E069E670E081E090E00E94A40406
:104C9000809152068330A9F48091370690913806AE
:104CA000019790933806809337060FE110E02CE3CC
:104CB00030E046EE50E069E670E081E090E00E946E
:104CC000A4048091370690913806039720F0109243
:104CD0003806109237068091370690913806813059
:104CE000910589F1D0F0029709F046C081E8E82EDD
:104CF00084E0F82E02E02FE130E04FEF5FEF6DE748
:104D000070E088E290E00E94990582E08093880636
:104D10004EE150E06AE570E02BC025E9E22E24E088
:104D2000F22E02E02FE130E04FEF5FEF6DE770E031
:104D300088E290E00E949905109288064EE150E0CA
:104D400066E970E015C09BE8E92E94E0F92E02E0D8
:104D50002FE130E04FEF5FEF6DE770E088E290E029
:104D60000E949905C09388064EE150E068E770E024
:104D700083E096E00E94CA478091520681110FC0DD
:104D8000A895C0935F0610923E0610923D06C09310
:104D90004D068FE190E00E941906A8950ED98091EA
:104DA0005206813059F5A89580935F0610923E0611
:104DB00010923D0680934D068FE190E00E94190607
:104DC000A8951092970680918806813069F038F096
:104DD000823091F44EE150E06AE570E009C04EE1A6
:104DE00050E066E970E004C04EE150E068E770E032
:104DF00083E096E00E94CA47A89513D0D09352064C
:104E00002FEF80E792E0215080409040E1F700C012
:104E100000001ECFDF91CF911F910F91FF90EF9077
:104E20000895EF92FF920F931F93CF93809197066F
:104E300081110C9415328FE190E00E9419060E94B6
:104E4000450D85E080935206C5E08091970681115B
:104E50000C9415320E94DD0C809152068230D9F4F8
:104E6000809183068F5F809383060FE110E02CE32F
:104E700030E046EE50E069E670E081E090E00E94AC
:104E8000A40422E330E043EC50E068E270E088E004
:104E900090E00E94A404809152068330D9F480915E
:104EA00083068150809383060FE110E02CE330E00D
:104EB00046EE50E069E670E081E090E00E94A404D4
:104EC00022E330E043EC50E068E270E088E090E0FC
:104ED0000E94A404809183068E3010F01092830605
:104EE000E09183068E2F90E08E30910510F00C94A7
:104EF000B830FC01E958FF4F80912C0690912D06A7
:104F00000C94BF44892BB9F5809103069091040657
:104F1000893E934020F010920406109203067BE332
:104F2000E72E74E0F72E01E02FE130E04FEF5FEF66
:104F300062E370E08FE090E00E949905E4E3EE2EDA
:104F4000E4E0FE2E2FE130E04FEF5FEF66E470E02B
:104F50008CE390E00E949905E0900306F09004062F
:104F600003E02FE130E04FEF5FEF62E870E080E5B3
:104F700090E00E94DF0580912C0690912D0601970C
:104F800009F0F1C78091030690910406893E934091
:104F900020F010920406109203065BE3E52E54E025
:104FA000F52E01E02FE130E04FEF5FEF62E370E0BC
:104FB0008FE090E00E94990564E3E62E64E0F62E0F
:104FC0002FE130E04FEF5FEF66E470E08CE390E0BC
:104FD0000E949905E0900306F0900406B9C7892B5A
:104FE000B9F58091050690910606893E934020F020
:104FF00010920606109205063CE1E32E34E0F32EF3
:1050000001E02FE130E04FEF5FEF62E370E08FE00F
:1050100090E00E9499054EE0E42E44E0F42E2FE14A
:1050200030E04FEF5FEF66E470E08CE390E00E94C9
:105030009905E0900506F090060603E02FE130E0C8
:105040004FEF5FEF62E870E080E590E00E94DF05DF
:1050500080912C0690912D068130910531F480913C
:1050600083068F5F8093830639C00297B9F58091DC
:10507000050690910606893E934020F010920606A0
:10508000109205069CE1E92E94E0F92E01E02FE153
:1050900030E04FEF5FEF62E370E08FE090E00E945E
:1050A00099052EE0E22E24E0F22E2FE130E04FEFC2
:1050B0005FEF66E470E08CE390E00E949905E09079
:1050C0000506F090060603E02FE130E04FEF5FEFBA
:1050D00062E870E080E590E00E94DF0580912C0698
:1050E00090912D060497B9F58091050690910606DA
:1050F000893E934020F010920606109205060CE1BE
:10510000E02E04E0F02E01E02FE130E04FEF5FEF02
:1051100062E370E08FE090E00E9499058EE0E82E57
:1051200084E0F82E2FE130E04FEF5FEF66E470E0AF
:105130008CE390E00E949905E0900506F090060649
:1051400003E02FE130E04FEF5FEF62E870E080E5D1
:1051500090E00E94DF0580912C0690912D06059726
:10516000B9F58091050690910606893E934020F09E
:105170001092060610920506BCE1EB2EB4E0FB2E61
:1051800001E02FE130E04FEF5FEF62E370E08FE08E
:1051900090E00E9499051EE0E12E14E0F12E2FE12F
:1051A00030E04FEF5FEF66E470E08CE390E00E9448
:1051B0009905E0900506F090060603E02FE130E047
:1051C0004FEF5FEF62E870E080E590E00E94DF055E
:1051D00080912C0690912D06069709F0C9C7809101
:1051E000050690910606893E934020F0109206062F
:1051F00010920506FCE1EF2EF4E0FF2E01E02FE116
:1052000030E04FEF5FEF62E370E08FE090E00E94EC
:105210009905AEE0EA2EA4E0FA2E2FE130E04FEF40
:105220005FEF66E470E08CE390E00E949905E09007
:105230000506F0900606E0C5892BB1F580910706BA
:10524000909108064F9720F01092080610920706DA
:1052500076EFE72E73E0F72E01E02FE130E04FEF1D
:105260005FEF62E370E08FE090E00E949905EEED61
:10527000EE2EE3E0FE2E2FE130E04FEF5FEF66E42D
:1052800070E08FE090E00E949905E0900706F090B2
:10529000080603E02FE130E04FEF5FEF62E870E0D7
:1052A00080E590E00E94DF0580912C0690912D060C
:1052B000019709F058C680910706909108064F970C
:1052C00020F0109208061092070656EFE52E53E0E4
:1052D000F52E01E02FE130E04FEF5FEF62E370E089
:1052E0008FE090E00E9499056EEDE62E63E0F62EC9
:1052F0002FE130E04FEF5FEF66E470E08FE090E089
:105300000E949905E0900706F090080621C6892BB7
:10531000B1F58091090690910A064F9720F01092FE
:105320000A061092090636ECE32E33E0F32E01E074
:105330002FE130E04FEF5FEF62E370E08FE090E04D
:105340000E9499054EEAE42E43E0F42E2FE130E06E
:105350004FEF5FEF66E470E08FE090E00E94990508
:10536000E0900906F0900A0603E02FE130E04FEFED
:105370005FEF62E870E080E590E00E94DF058091D9
:105380002C0690912D068130910531F48091830691
:105390008F5F8093830638C00297B1F5809109062C
:1053A00090910A064F9720F010920A061092090673
:1053B00096ECE92E93E0F92E01E02FE130E04FEF7B
:1053C0005FEF62E370E08FE090E00E9499052EEAC3
:1053D000E22E23E0F22E2FE130E04FEF5FEF66E4A4
:1053E00070E08FE090E00E949905E0900906F0904F
:1053F0000A0603E02FE130E04FEF5FEF62E870E074
:1054000080E590E00E94DF0580912C0690912D06AA
:105410000497B1F58091090690910A064F9720F004
:1054200010920A061092090606ECE02E03E0F02E18
:1054300001E02FE130E04FEF5FEF62E370E08FE0DB
:1054400090E00E9499058EEAE82E83E0F82E2FE185
:1054500030E04FEF5FEF66E470E08FE090E00E9495
:105460009905E0900906F0900A0603E02FE130E08C
:105470004FEF5FEF62E870E080E590E00E94DF05AB
:1054800080912C0690912D060597B1F58091090623
:1054900090910A064F9720F010920A061092090682
:1054A000B6ECEB2EB3E0FB2E01E02FE130E04FEF46
:1054B0005FEF62E370E08FE090E00E9499051EEAE2
:1054C000E12E13E0F12E2FE130E04FEF5FEF66E4C5
:1054D00070E08FE090E00E949905E0900906F0905E
:1054E0000A0603E02FE130E04FEF5FEF62E870E083
:1054F00080E590E00E94DF0580912C0690912D06BA
:10550000069709F035C68091090690910A064F97D3
:1055100020F010920A0610920906F6ECEF2EF3E046
:10552000FF2E01E02FE130E04FEF5FEF62E370E02C
:105530008FE090E00E949905AEEAEA2EA3E0FA2EF1
:105540002FE130E04FEF5FEF66E470E08FE090E036
:105550000E949905E0900906F0900A064DC4892B37
:1055600009F045C080910B0690910C06039730F02E
:1055700081E090E090930C0680930B06E6E9EE2E16
:10558000E3E0FE2E01E02FE130E04FEF5FEF6CE350
:1055900070E08FE090E00E94990580910B06909159
:1055A0000C06019779F473E5E72E75E0F72E03E01A
:1055B0002FE130E04FEF5FEF62E870E080E590E0D0
:1055C0000E94990580910B0690910C06892B79F425
:1055D0006EE4E62E65E0F62E03E02FE130E04FEFBB
:1055E0005FEF62E870E080E590E00E9499058091AD
:1055F0002C0690912D068130910509F044C0209130
:105600000B0630910C062330310520F090930C06E8
:1056100080930B0656E9E52E53E0F52E01E02FE1CD
:1056200030E04FEF5FEF6CE370E08FE090E00E94BE
:10563000990580910B0690910C06019779F443E54A
:10564000E42E45E0F42E03E02FE130E04FEF5FEF72
:1056500062E870E080E590E00E94990580910B0679
:1056600090910C06892B79F43EE4E32E35E0F32E7D
:1056700003E02FE130E04FEF5FEF62E870E080E59C
:1056800090E00E94990580912C0690912D0602973A
:1056900009F045C080910B0690910C06039730F0FD
:1056A00081E090E090930C0680930B0626E9E22EB1
:1056B00023E0F22E01E02FE130E04FEF5FEF6CE3EB
:1056C00070E08FE090E00E94990580910B06909128
:1056D0000C06019779F493E5E92E95E0F92E03E0A5
:1056E0002FE130E04FEF5FEF62E870E080E590E09F
:1056F0000E94990580910B0690910C06892B79F4F4
:105700008EE4E82E85E0F82E03E02FE130E04FEF45
:105710005FEF62E870E080E590E00E94990580917B
:105720002C0690912D069C01245031092230310520
:1057300008F4D9C4069709F01BC580910B06909117
:105740000C06039730F081E090E090930C06809374
:105750000B0606E9E02E03E0F02E01E02FE130E039
:105760004FEF5FEF6CE370E08FE090E00E949905EF
:1057700080910B0690910C06019779F413E5E12EC8
:1057800015E0F12E03E02FE130E04FEF5FEF62E82C
:1057900070E080E590E00E94990580910B06909161
:1057A0000C06892B09F0E4C4BEE4EB2EB5E0FB2E19
:1057B00003E02FE130E04FEF5FEF62E870E080E55B
:1057C00090E00E949905D4C4892BB9F580910D060B
:1057D00090910E068F35914020F010920E06109297
:1057E0000D06FEE7EF2EF3E0FF2E01E02FE130E0A3
:1057F0004FEF5FEF62E370E08FE090E00E94990569
:10580000A6E6EA2EA3E0FA2E2FE130E04FEF5FEF9D
:1058100066E470E08FE090E00E949905E0900D064C
:10582000F0900E0603E02FE130E04FEF5FEF62E80B
:1058300070E080E590E00E94DF0580912C06909159
:105840002D060197B9F580910D0690910E068F35C2
:10585000914020F010920E0610920D067EE7E72E82
:1058600073E0F72E01E02FE130E04FEF5FEF62E3EE
:1058700070E08FE090E00E949905E6E6EE2EE3E00E
:10588000FE2E2FE130E04FEF5FEF66E470E08FE037
:1058900090E00E949905E0900D06F0900E0603E05E
:1058A0002FE130E04FEF5FEF62E870E080E590E0DD
:1058B0000E94DF0580912C0690912D060297B9F584
:1058C00080910D0690910E068F35914020F0109238
:1058D0000E0610920D065EE7E52E53E0F52E01E070
:1058E0002FE130E04FEF5FEF62E370E08FE090E098
:1058F0000E94990566E6E62E63E0F62E2FE130E081
:105900004FEF5FEF66E470E08FE090E00E94990552
:10591000E0900D06F0900E0603E02FE130E04FEF2F
:105920005FEF62E870E080E590E00E94DF05809123
:105930002C0690912D069C0124503109223031050E
:1059400008F4D1C3069709F013C480910D06909115
:105950000E068F35914020F010920E0610920D0623
:105960003EE7E32E33E0F32E01E02FE130E04FEF8E
:105970005FEF62E370E08FE090E00E94990546E6F9
:10598000E42E43E0F42E2FE130E04FEF5FEF66E4CA
:1059900070E08FE090E00E949905E0900D06F09095
:1059A0000E062AC2892BB9F580910F069091100638
:1059B0008636910520F01092100610920F069EE494
:1059C000E92E93E0F92E01E02FE130E04FEF5FEF99
:1059D00062E370E08FE090E00E94990526E3E22EFA
:1059E00023E0F22E2FE130E04FEF5FEF66E470E04E
:1059F0008FE090E00E949905E0900F06F09010066D
:105A000003E02FE130E04FEF5FEF62E870E080E508
:105A100090E00E94DF0580912C0690912D06019761
:105A2000B9F580910F06909110068636910520F009
:105A30001092100610920F060EE4E02E03E0F02EF6
:105A400001E02FE130E04FEF5FEF62E370E08FE0C5
:105A500090E00E94990586E3E82E83E0F82E2FE17E
:105A600030E04FEF5FEF66E470E08FE090E00E947F
:105A70009905E0900F06F090100603E02FE130E06A
:105A80004FEF5FEF62E870E080E590E00E94DF0595
:105A900080912C0690912D068230910531F48091F1
:105AA00083068F5F8093830639C00497B9F5809190
:105AB0000F06909110068636910520F01092100680
:105AC00010920F06BEE4EB2EB3E0FB2E01E02FE1B7
:105AD00030E04FEF5FEF62E370E08FE090E00E9414
:105AE000990516E3E12E13E0F12E2FE130E04FEFA0
:105AF0005FEF66E470E08FE090E00E949905E0902F
:105B00000F06F090100603E02FE130E04FEF5FEF5B
:105B100062E870E080E590E00E94DF0580912C064D
:105B200090912D060597B9F580910F06909110067A
:105B30008636910520F01092100610920F06FEE4B2
:105B4000EF2EF3E0FF2E01E02FE130E04FEF5FEFAB
:105B500062E370E08FE090E00E949905A6E3EA2EF0
:105B6000A3E0FA2E2FE130E04FEF5FEF66E470E044
:105B70008FE090E00E949905E0900F06F0901006EB
:105B800003E02FE130E04FEF5FEF62E870E080E587
:105B900090E00E94DF0580912C0690912D06A0C216
:105BA000892BB9F5809111069091120686369105E0
:105BB00020F010921206109211067EE1E72E73E09B
:105BC000F72E01E02FE130E04FEF5FEF62E370E08E
:105BD0008FE090E00E949905E6E0EE2EE3E0FE2ED5
:105BE0002FE130E04FEF5FEF66E470E08FE090E090
:105BF0000E949905E0901106F090120603E02FE153
:105C000030E04FEF5FEF62E870E080E590E00E94E7
:105C1000DF0580912C0690912D068130910531F49D
:105C2000809183068F5F8093830639C00297B9F510
:105C300080911106909112068636910520F01092FF
:105C40001206109211065EE1E52E53E0F52E01E0FA
:105C50002FE130E04FEF5FEF62E370E08FE090E024
:105C60000E94990566E0E62E63E0F62E2FE130E013
:105C70004FEF5FEF66E470E08FE090E00E949905DF
:105C8000E0901106F090120603E02FE130E04FEFB4
:105C90005FEF62E870E080E590E00E94DF058091B0
:105CA0002C0690912D060497B9F5809111069091DC
:105CB00012068636910520F01092120610921106F7
:105CC0003EE1E32E33E0F32E01E02FE130E04FEF31
:105CD0005FEF62E370E08FE090E00E94990546E09C
:105CE000E42E43E0F42E2FE130E04FEF5FEF66E467
:105CF00070E08FE090E00E949905E0901106F0902E
:105D0000120603E02FE130E04FEF5FEF62E870E052
:105D100080E590E00E94DF0580912C0690912D0691
:105D20000597B9F580911106909112068636910576
:105D300020F010921206109211069EE1E92E93E0D7
:105D4000F92E01E02FE130E04FEF5FEF62E370E00A
:105D50008FE090E00E94990526E0E22E23E0F22EEB
:105D60002FE130E04FEF5FEF66E470E08FE090E00E
:105D70000E949905E0901106F090120603E02FE1D1
:105D800030E04FEF5FEF62E870E080E590E00E9466
:105D9000DF0580912C0690912D06069709F0E8C149
:105DA00080911106909112068636910520F010928E
:105DB0001206109211061EE1E12E13E0F12E01E011
:105DC0002FE130E04FEF5FEF62E370E08FE090E0B3
:105DD0000E94990586E0E82E83E0F82E2FE130E05E
:105DE0004FEF5FEF66E470E08FE090E00E9499056E
:105DF000E0901106F090120603E02FE130E04FEF43
:105E00005FEF62E870E080E590E00E94DF05B0C1DE
:105E1000892B49F580911B0690911C068D3291408B
:105E200020F010921C0610921B06B6E8EB2EB2E092
:105E3000FB2E01E02FE130E04FEF5FEF6CE370E00D
:105E40008FE090E00E949905E0901B06F0901C0600
:105E500003E02FE130E04FEF5FEF62E870E080E5B4
:105E600090E00E94DF0580912C0690912D0601970D
:105E700009F079C080911B0690911C068D329140EB
:105E800020F010921C0610921B06A6E8EA2EA2E053
:105E9000FA2E01E02FE130E04FEF5FEF6CE370E0AE
:105EA0008FE090E00E949905E0901B06F0901C06A0
:105EB0004FC0892B49F580911D0690911E06893EA1
:105EC000934020F010921E0610921D06FCEDEF2E5E
:105ED000F2E0FF2E01E02FE130E04FEF5FEF6CE3E7
:105EE00070E08FE090E00E949905E0901D06F09030
:105EF0001E0603E02FE130E04FEF5FEF62E870E055
:105F000080E590E00E94DF0580912C0690912D069F
:105F1000019749F580911D0690911E06893E934098
:105F200020F010921E0610921D06ECEDEE2EE2E01F
:105F3000FE2E01E02FE130E04FEF5FEF6CE370E009
:105F40008FE090E00E949905E0901D06F0901E06FB
:105F500003E02FE130E04FEF5FEF62E870E080E5B3
:105F600090E00E94DF0580912C0690912D068230F2
:105F7000910509F4B8C09C01245031092230310543
:105F800008F0AEC0B0C0892B09F094C08091130610
:105F900090911406039720F01092140610921306A5
:105FA00074EFE72E72E0F72E01E02FE130E04FEFC3
:105FB0005FEF6CE370E08EE190E00E9499058091C4
:105FC000130690911406019779F463E5E62E65E0D7
:105FD000F62E03E02FE130E04FEF5FEF62E870E074
:105FE00080E590E00E949905809113069091140637
:105FF000892B79F45EE4E52E55E0F52E03E02FE1E0
:1060000030E04FEF5FEF62E870E080E590E00E94E3
:106010009905809113068093F2054CC0892B09F0F5
:1060200049C08091F20581110BC01092830653C0C4
:10603000892B09F03FC08091F205811149C0F5CF4D
:10604000813009F048C08091150690911606893E6E
:10605000934020F010921606109215063EE7E32EAC
:1060600033E0F32E01E02FE130E04FEF5FEF62E32A
:1060700070E08FE090E00E94990546ECE42E42E04B
:10608000F42E2FE130E04FEF5FEF66E470E08FE039
:1060900090E00E949905E0901506F090160603E046
:1060A0002FE130E04FEF5FEF62E870E080E590E0D5
:1060B0000E94DF0580912C0690912D06813091057C
:1060C00091F08230910579F08430910561F005C03E
:1060D000813009F47DC180E090E08530910519F0B0
:1060E000069709F045C0809183068F5F80938306F1
:1060F0003FC0009731F09C01215031092230310519
:1061000018F4109283062BC0049749F580911F065E
:1061100090912006893E934020F010922006109224
:106120001F068FE5E82E82E0F82E01E02FE130E037
:106130004FEF5FEF6CE370E08FE090E00E94990515
:10614000E0901F06F090200603E02FE130E04FEFD3
:106150005FEF62E870E080E590E00E94DF058091EB
:106160002C0690912D060597029710F41092830645
:1061700080915206813009F00EC1809397061092EB
:106180005F0680912C0690912D06892B41F5E091B8
:106190003706F0913806E830F10508F5EB57FF4F68
:1061A0004EE150E00C94BF4464E972E014C066E72D
:1061B00072E011C068E572E00EC06AE372E00BC0E5
:1061C0006CE172E008C06EEF71E005C060EE71E056
:1061D00002C062EC71E083E096E00E94E7478091A4
:1061E0002C0690912D060197E1F48091370690914D
:1061F00038068130910569F038F0029791F44EE14C
:1062000050E068E671E009C04EE150E064EA71E0F8
:1062100004C04EE150E066E871E083E096E00E9441
:10622000E74780912C0690912D060297E1F480912A
:106230003706909138068130910569F038F0029761
:1062400091F44EE150E06EE071E009C04EE150E0A3
:106250006AE471E004C04EE150E06CE271E083E07A
:1062600096E00E94E74780912C0690912D060497B6
:10627000E1F480913706909138068130910569F0FC
:1062800038F0029791F44EE150E064EB70E009C001
:106290004EE150E060EF70E004C04EE150E062ED8E
:1062A00070E083E096E00E94E74780912C06909191
:1062B0002D060597E1F480913706909138068130DC
:1062C000910569F038F0029791F44EE150E06AE5EB
:1062D00070E009C04EE150E066E970E004C04EE1B4
:1062E00050E068E770E083E096E00E94E747809125
:1062F0002C0690912D060697E1F480913706909137
:1063000038068130910569F038F0029791F44EE13A
:1063100050E060E070E009C04EE150E06CE370E0F6
:1063200004C04EE150E06EE170E083E096E00E9430
:10633000E7478FE190E00E94190680912C0690912A
:106340002D06892B09F47FD180912C0690912D0682
:10635000019711F40E94BF3B80912C0690912D066D
:10636000029711F40E94C63C80912C0690912D0654
:10637000049711F40E94CD3D80912C0690912D063A
:10638000059711F40E940B2680912C0690912D0602
:10639000069709F450D08091520681110CC081E01B
:1063A0008093970610925F06109221068FE190E08D
:1063B0000E941906EBD2C09352068FE798E321E0C2
:1063C000815090402040E1F700C000000C94252748
:1063D0008091170690911806893E934020F0109204
:1063E0001806109217069FEAE92E92E0F92E01E0B6
:1063F0002FE130E04FEF5FEF62E370E08FE090E07D
:106400000E9499052CE9E22E22E0F22E2FE130E0E5
:106410004FEF5FEF66E470E08FE090E00E94990537
:10642000E0901706F09018063ACECF911F910F9189
:10643000FF90EF900895EF92FF920F931F93CF93E9
:10644000DF93A89580915F068111F6C08FE190E0FF
:106450000E9419060E944F0C8091850690E090934F
:1064600038068093370685E080935206C1E0D5E078
:1064700080915F068111E0C0A8950E94DD0C80919B
:1064800052068230A9F48091370690913806019621
:1064900090933806809337060FE110E02CE330E04C
:1064A00046EE50E069E670E081E090E00E94A404CE
:1064B000809152068330A9F4809137069091380676
:1064C000019790933806809337060FE110E02CE394
:1064D00030E046EE50E069E670E081E090E00E9436
:1064E000A4048091370690913806039720F010920B
:1064F0003806109237068091370690913806813021
:10650000910589F1D0F0029709F046C081E8E82EA4
:1065100084E0F82E02E02FE130E04FEF5FEF6DE70F
:1065200070E088E290E00E94990582E08093850601
:106530004EE150E060E070E02BC025E9E22E24E05F
:10654000F22E02E02FE130E04FEF5FEF6DE770E0F9
:1065500088E290E00E949905109285064EE150E095
:106560006CE370E015C09BE8E92E94E0F92E02E0A0
:106570002FE130E04FEF5FEF6DE770E088E290E0F1
:106580000E949905C09385064EE150E06EE170E0EF
:1065900083E096E00E94CA4780915206811110C0A4
:1065A000A895C0935F0610923E0610923D06C093D8
:1065B0004D068FE190E00E941906A8950E94DD1F0C
:1065C00080915206813061F5A89580935F06109204
:1065D0003E0610923D0680934D068FE190E00E94AA
:1065E0001906A8951092970680918506813069F06A
:1065F00038F0823091F44EE150E060E070E009C084
:106600004EE150E06CE370E004C04EE150E06EE11A
:1066100070E083E096E00E94CA47A8950E94112787
:10662000D09352062FEF80E792E0215080409040B7
:10663000E1F700C000001CCFDF91CF911F910F91B7
:10664000FF90EF900895AF92BF92CF92DF92EF92BA
:10665000FF920F931F93CF93DF93A89580915F06CE
:10666000811189C18FE190E00E9419060E944F0CB0
:106670008091890690E0909338068093370685E0F4
:1066800080935206E7E0DE2EF6E0CF2ED5E0A4E0C0
:10669000BA2EB3E0AB2EC1E080915F0681116BC1D1
:1066A000A8950E94DD0C809152068230A9F4809159
:1066B00037069091380601969093380680933706F6
:1066C0000FE110E02CE330E046EE50E069E670E0C8
:1066D00081E090E00E94A404809152068330A9F4E6
:1066E00080913706909138060197909338068093F1
:1066F00037060FE110E02CE330E046EE50E069E6AB
:1067000070E081E090E00E94A404809137069091AF
:106710003806089720F01092380610923706E0915C
:106720003706F0913806E830F10508F0BEC0E357AF
:10673000FF4F0C94BF4474EAE72E74E0F72E02E09A
:106740002FE130E04FEF5FEF6DE770E082E390E024
:106750000E949905109289064EE150E064E972E0CA
:106760009AC06FE9E62E64E0F62E02E02FE130E0F9
:106770004FEF5FEF6DE770E082E390E00E949905D4
:10678000C09389064EE150E066E772E084C055E9A7
:10679000E52E54E0F52E02E02FE130E04FEF5FEF01
:1067A0006DE770E088E290E00E94990582E08093B6
:1067B00089064EE150E068E572E06DC04BE8E42EDA
:1067C00044E0F42E02E02FE130E04FEF5FEF6DE7A1
:1067D00070E088E290E00E949905A09289064EE15F
:1067E00050E06AE372E057C031E8E32E34E0F32E64
:1067F00002E02FE130E04FEF5FEF6DE770E088E2FD
:1068000090E00E949905B092890644E150E06CE165
:1068100072E041C027E7E22E24E0F22E02E02FE1F1
:1068200030E04FEF5FEF6DE770E088E290E00E94AC
:106830009905D09389064EE150E06EEF71E02BC0D0
:106840009DE6E92E94E0F92E02E02FE130E04FEFD3
:106850005FEF6DE770E088E290E00E949905C092DA
:1068600089064EE150E060EE71E015C083E6E82E47
:1068700084E0F82E02E02FE130E04FEF5FEF6DE7AC
:1068800070E088E290E00E949905D09289064EE17E
:1068900050E062EC71E083E096E00E94CA478FE529
:1068A0009AEE0197F1F700C0000080915206811125
:1068B0000FC0A895C0935F0610923E0610923D0649
:1068C000C0934D068FE190E00E9419060E94DD1FE3
:1068D00080915206813009F041C0A89580935F06EF
:1068E00010923E0610923D0680934D068FE190E097
:1068F0000E94190610929706E09189068E2F90E06B
:106900008830910540F5FC01EB56FF4F4EE150E019
:106910000C94BF4464E972E014C066E772E011C0F1
:1069200068E572E00EC06AE372E00BC06CE172E0F1
:1069300008C06EEF71E005C060EE71E002C062EC6D
:1069400071E083E096E00E94CA478FE59AEE0197D6
:10695000F1F700C00000A8950E941127D0935206BD
:10696000A8959FEF20E782E0915020408040E1F71A
:1069700000C0000091CEDF91CF911F910F91FF9049
:10698000EF90DF90CF90BF90AF900895BF92CF92DD
:10699000DF92EF92FF920F931F93CF93DF9380913B
:1069A00021068111E2C68FE190E00E9419060E9443
:1069B000450D1092840685E08093520698E5C92E15
:1069C00092E0D92ECAE5D0E025E0B22E80912106D2
:1069D0008111CBC6E09183068E2F90E08E30910519
:1069E00008F0B2C6FC01E356FF4F0C94BF441BE312
:1069F000E12E14E0F12E01E02FE130E04FEF5FEFE8
:106A000062E370E08FE090E00E94990584E3E82E55
:106A100084E0F82E2FE130E04FEF5FEF66E470E0A6
:106A20008CE390E00E949905E0900306F090040644
:106A300003E02FE130E040E058EF62E870E080E5ED
:106A400090E00E94DF0580910306909104069093E8
:106A5000F7058093F6050E94DD0C80915206823086
:106A6000A9F48091F6059091F70501969093F705AA
:106A70008093F6050FE110E02CE330E046EE50E0A5
:106A800069E670E081E090E00E94A40480915206E3
:106A90008330A9F48091F6059091F70501979093C2
:106AA000F7058093F6050FE110E02CE330E046EEA9
:106AB00050E069E670E081E090E00E94A4048091DB
:106AC000F6059091F7058F35914020F01092F7056B
:106AD0001092F6058091F6059091F70590930406C3
:106AE0008093030628C6ACE1EA2EA4E0FA2E01E06A
:106AF0002FE130E04FEF5FEF62E370E08FE090E076
:106B00000E949905BEE0EB2EB4E0FB2E2FE130E0B1
:106B10004FEF5FEF66E470E08CE390E00E94990530
:106B2000E0900506F090060603E02FE130E040E03B
:106B300058EF62E870E080E590E00E94DF05809108
:106B400005069091060690934A06809349060E9496
:106B5000DD0C809152068230A9F480914906909113
:106B60004A06019690934A06809349060FE110E089
:106B70002CE330E046EE50E069E670E081E090E022
:106B80000E94A404809152068330A9F480914906A2
:106B900090914A06019790934A06809349060FE127
:106BA00010E02CE330E046EE50E069E670E081E072
:106BB00090E00E94A4048091490690914A06853F86
:106BC000914020F010924A061092490680914906A1
:106BD00090914A069093060680930506ACC5E6EFB1
:106BE000EE2EE3E0FE2E01E02FE130E04FEF5FEF0D
:106BF00062E370E08FE090E00E949905FEEDEF2ED9
:106C0000F3E0FF2E2FE130E04FEF5FEF66E470E03E
:106C10008FE090E00E949905E0900706F09008064A
:106C200003E02FE130E040E058EF62E870E080E5FB
:106C300090E00E94DF0580910706909108069093EE
:106C40009206809391060E94DD0C8091520682305C
:106C5000A9F48091910690919206019690939206E4
:106C6000809391060FE110E02CE330E046EE50E017
:106C700069E670E081E090E00E94A40480915206F1
:106C80008330A9F480919106909192060197909398
:106C90009206809391060FE110E02CE330E046EE7F
:106CA00050E069E670E081E090E00E94A4048091E9
:106CB0009106909192064F9730F08FE090E090937C
:106CC00092068093910680919106909192060F977B
:106CD00030F48FE090E0909392068093910680913B
:106CE000910690919206909308068093070623C51B
:106CF00066ECE62E63E0F62E01E02FE130E04FEF88
:106D00005FEF62E370E08FE090E00E9499057EEA19
:106D1000E72E73E0F72E2FE130E04FEF5FEF66E4F0
:106D200070E08FE090E00E949905E0900906F090F5
:106D30000A0603E02FE130E040E058EF62E870E03F
:106D400080E590E00E94DF058091090690910A0697
:106D500090933406809333060E94DD0C8091520696
:106D60008230A9F480913306909134060196909375
:106D70003406809333060FE110E02CE330E046EE5A
:106D800050E069E670E081E090E00E94A404809108
:106D900052068330A9F4809133069091340601970E
:106DA00090933406809333060FE110E02CE330E03B
:106DB00046EE50E069E670E081E090E00E94A404B5
:106DC00080913306909134064F9730F08FE090E039
:106DD0009093340680933306809133069091340665
:106DE0000F9730F48FE090E0909334068093330651
:106DF000809133069091340690930A068093090699
:106E00009AC456E9E52E53E0F52E01E02FE130E07B
:106E10004FEF5FEF6CE370E08FE090E00E94990528
:106E200080910B0690910C06019779F443E5E42ECE
:106E300045E0F42E03E02FE130E040E058EF62E857
:106E400070E080E590E00E94990580910B0690919A
:106E50000C06892B79F43EE4E32E35E0F32E03E0B3
:106E60002FE130E040E058EF62E870E080E590E02C
:106E70000E94990580910B0680935E060E94DD0CAE
:106E800080915206823089F480915E068F5F8093F4
:106E90005E060FE110E02CE330E046EE50E069E6DC
:106EA00070E081E090E00E94A4048091520683305B
:106EB00089F480915E06815080935E060FE110E0B8
:106EC0002CE330E046EE50E069E670E081E090E0CF
:106ED0000E94A40480915E06823010F010925E063B
:106EE00080915E0690E090930C0680930B0623C47D
:106EF0009EE7E92E93E0F92E01E02FE130E04FEF1D
:106F00005FEF62E370E08FE090E00E94990526E673
:106F1000E22E23E0F22E2FE130E04FEF5FEF66E448
:106F200070E08FE090E00E949905E0900D06F090EF
:106F30000E0603E020E038EF4FEF5FEF62E870E00D
:106F400080E590E00E94DF0580910D0690910E068D
:106F500090933206809331060E94DD0C8091520698
:106F60008230A9F480913106909132060196909377
:106F70003206809331060FE110E02CE330E046EE5C
:106F800050E069E670E081E090E00E94A404809106
:106F900052068330A9F48091310690913206019710
:106FA00090933206809331060FE110E02CE330E03D
:106FB00046EE50E069E670E081E090E00E94A404B3
:106FC00080913106909132068B3F910520F010920E
:106FD00032061092310680913106909132069093DC
:106FE0000E0680930D06A7C31EE4E12E13E0F12EDA
:106FF00001E02FE130E04FEF5FEF62E370E08FE000
:1070000090E00E94990586E3E82E83E0F82E2FE1B8
:1070100030E04FEF5FEF66E470E08FE090E00E94B9
:107020009905E0900F06F090100603E02FE130E0A4
:1070300040E058EF62E870E080E590E00E94DF05F4
:1070400080910F06809342060E94DD0C80915206CB
:10705000823089F4809142068F5F809342060FE16F
:1070600010E02CE330E046EE50E069E670E081E0AD
:1070700090E00E94A40480915206833089F48091AC
:1070800042068150809342060FE110E02CE330E08D
:1070900046EE50E069E670E081E090E00E94A404D2
:1070A00080914206853610F0109242068091420689
:1070B00090E09093100680930F063DC3AEE1EA2E58
:1070C000A3E0FA2E01E02FE130E04FEF5FEF62E343
:1070D00070E08FE090E00E949905B6E0EB2EB3E0FF
:1070E000FB2E2FE130E04FEF5FEF66E470E08FE0C2
:1070F00090E00E949905E0901106F090120603E0DE
:107100002FE130E040E058EF62E870E080E590E089
:107110000E94DF0580911106809341060E94DD0CDC
:1071200080915206823089F4809141068F5F80936E
:1071300041060FE110E02CE330E046EE50E069E656
:1071400070E081E090E00E94A404809152068330B8
:1071500089F4809141068150809341060FE110E04F
:107160002CE330E046EE50E069E670E081E090E02C
:107170000E94A40480914106853610F010924106C9
:107180008091410690E09093120680931106D3C23D
:10719000F6E8EF2EF2E0FF2E01E02FE130E04FEFB6
:1071A0005FEF6CE370E08FE090E00E949905E09063
:1071B0001B06F0901C0603E02FE130E040E058EFA2
:1071C00062E870E080E590E00E94DF0580911B0698
:1071D00090911C069093800680937F060E94DD0CA0
:1071E000809152068230A9F480917F0690918006AA
:1071F00001969093800680937F060FE110E02CE3C8
:1072000030E046EE50E069E670E081E090E00E94F8
:10721000A404809152068330A9F480917F06909156
:10722000800601979093800680937F060FE110E01F
:107230002CE330E046EE50E069E670E081E090E05B
:107240000E94A40480917F0690918006893C91055C
:1072500020F0D0938006C0937F0680917F069091A6
:1072600080068A35910520F4D0938006C0937F066E
:1072700080917F069091800690931C0680931B0658
:107280005AC2ECEDEE2EE2E0FE2E01E02FE130E0FE
:107290004FEF5FEF6CE370E08FE090E00E949905A4
:1072A000E0901D06F0901E0603E02FE130E040E084
:1072B00058EF62E870E080E590E00E94DF05809181
:1072C0001D0690911E0690930206809301060E946F
:1072D000DD0C809152068230A9F4809101069091D4
:1072E0000206019690930206809301060FE110E0DA
:1072F0002CE330E046EE50E069E670E081E090E09B
:107300000E94A404809152068330A9F48091010662
:1073100090910206019790930206809301060FE177
:1073200010E02CE330E046EE50E069E670E081E0EA
:1073300090E00E94A4048091010690910206C397F8
:1073400020F01092020610920106809101069091A1
:10735000020690931E0680931D06EDC174EFE72E82
:1073600072E0F72E01E02FE130E04FEF5FEF6CE3CA
:1073700070E08EE190E00E94990580911306909153
:107380001406019779F463E5E62E65E0F62E03E036
:107390002FE130E040E058EF62E870E080E590E0F7
:1073A0000E9499058091130690911406892B79F417
:1073B0005EE4E52E55E0F52E03E02FE130E040E0FD
:1073C00058EF62E870E080E590E00E9499058091B6
:1073D00013068093F2050E94DD0C809152068230E4
:1073E00089F48091F2058F5F8093F2050FE110E040
:1073F0002CE330E046EE50E069E670E081E090E09A
:107400000E94A40480915206833089F48091F20591
:1074100081508093F2050FE110E02CE330E046EE5E
:1074200050E069E670E081E090E00E94A404809161
:10743000F205823010F01092F2058091F20590E092
:10744000909314068093130676C18091F205811102
:1074500003C01092830678C1813009F075C13EE700
:10746000E32E33E0F32E01E02FE130E04FEF5FEF4A
:1074700062E370E08FE090E00E94990546ECE42E14
:1074800042E0F42E2FE130E04FEF5FEF66E470E072
:107490008FE090E00E949905E0901506F0901606A6
:1074A00003E02FE130E040E058EF62E870E080E573
:1074B00090E00E94DF05809115069091160690934A
:1074C0008206809381060E94DD0C809152068230F4
:1074D000A9F480918106909182060196909382068C
:1074E000809381060FE110E02CE330E046EE50E09F
:1074F00069E670E081E090E00E94A4048091520669
:107500008330A9F48091810690918206019790932F
:107510008206809381060FE110E02CE330E046EE16
:1075200050E069E670E081E090E00E94A404809160
:107530008106909182068B3F910520F01092820681
:107540001092810680918106909182069093160692
:1075500080931506F0C08091F205882309F479CF55
:10756000813009F0F1C09FEAE92E92E0F92E01E0A6
:107570002FE130E04FEF5FEF62E370E08FE090E0EB
:107580000E9499052CE9E22E22E0F22E2FE130E054
:107590004FEF5FEF66E470E08FE090E00E949905A6
:1075A000E0901706F090180603E02FE130E040E08D
:1075B00058EF62E870E080E590E00E94DF0580917E
:1075C00017069091180690935D0680935C060E94C2
:1075D000DD0C809152068230A9F480915C06909176
:1075E0005D06019690935D0680935C060FE110E0C6
:1075F0002CE330E046EE50E069E670E081E090E098
:107600000E94A404809152068330A9F480915C0604
:1076100090915D06019790935D0680935C060FE163
:1076200010E02CE330E046EE50E069E670E081E0E7
:1076300090E00E94A40480915C0690915D06C3973F
:1076400020F010925D0610925C0680915C0690918D
:107650005D0690931806809317066DC08FE5E82E9F
:1076600082E0F82E01E02FE130E04FEF5FEF6CE3B6
:1076700070E08FE090E00E949905E0901F06F09086
:10768000200603E02FE130E040E058EF62E870E0D0
:1076900080E590E00E94DF0580911F069091200612
:1076A00090932706809326060E94DD0C8091520657
:1076B0008230A9F480912606909127060196909336
:1076C0002706809326060FE110E02CE330E046EE1B
:1076D00050E069E670E081E090E00E94A4048091AF
:1076E00052068330A9F480912606909127060197CF
:1076F00090932706809326060FE110E02CE330E0FC
:1077000046EE50E069E670E081E090E00E94A4045B
:1077100080910106909102068935924020F0D09226
:107720002706C09226068091260690912706909300
:10773000200680931F068FE798E321E08150904058
:107740002040E1F700C0000080915206813051F4E2
:1077500080932106109297068FE190E00E9419060F
:107760000E941127B092520631C9DF91CF911F912B
:107770000F91FF90EF90DF90CF90BF900895EF9220
:10778000FF920F931F93CF93DF93A89580915F068D
:107790008111F5C08FE190E00E9419060E944F0C04
:1077A0008091350690E0909338068093370685E007
:1077B00080935206C1E0D5E080915F068111DFC061
:1077C000A8950E94DD0C809152068230A9F4809128
:1077D00037069091380601969093380680933706C5
:1077E0000FE110E02CE330E046EE50E069E670E097
:1077F00081E090E00E94A404809152068330A9F4B5
:1078000080913706909138060197909338068093BF
:1078100037060FE110E02CE330E046EE50E069E679
:1078200070E081E090E00E94A4048091370690917E
:107830003806039720F01092380610923706A89564
:1078400080913706909138068130910589F1D0F00A
:10785000029709F046C081E8E82E84E0F82E02E0A5
:107860002FE130E04FEF5FEF6DE770E088E290E0EE
:107870000E94990582E0809335064EE150E068E66B
:1078800071E02BC025E9E22E24E0F22E02E02FE188
:1078900030E04FEF5FEF6DE770E088E290E00E942C
:1078A0009905109235064EE150E064EA71E015C08A
:1078B0009BE8E92E94E0F92E02E02FE130E04FEF53
:1078C0005FEF6DE770E088E290E00E949905C09359
:1078D00035064EE150E066E871E083E096E00E94F4
:1078E000CA478091520681110FC0A895C0935F06C8
:1078F00010923E0610923D06C0934D068FE190E037
:107900000E9419060E94DD1F80915206813059F5B0
:10791000A89580935F0610923E0610923D068093D4
:107920004D068FE190E00E94190610929706809113
:107930003506813069F038F0823091F44EE150E044
:1079400068E671E009C04EE150E064EA71E004C00D
:107950004EE150E066E871E083E096E00E94CA479D
:10796000A8950E941127D09352062FEF80E792E04E
:10797000215080409040E1F700C000001DCFDF9112
:10798000CF911F910F91FF90EF900895EF92FF928A
:107990000F931F93CF93DF93A89580915F0681117A
:1079A000F5C08FE190E00E9419060E944F0C809173
:1079B0003C0690E0909338068093370685E08093EC
:1079C0005206C1E0D5E080915F068111DFC0A89525
:1079D0000E94DD0C809152068230A9F48091370616
:1079E00090913806019690933806809337060FE100
:1079F00010E02CE330E046EE50E069E670E081E014
:107A000090E00E94A404809152068330A9F48091F2
:107A10003706909138060197909338068093370681
:107A20000FE110E02CE330E046EE50E069E670E054
:107A300081E090E00E94A40480913706909138067E
:107A4000039720F01092380610923706809137067F
:107A5000909138068130910589F1D0F0029709F0B4
:107A600046C081E8E82E84E0F82E02E02FE130E005
:107A70004FEF5FEF6DE770E088E290E00E949905BC
:107A800082E080933C064EE150E06EE071E02BC056
:107A900025E9E22E24E0F22E02E02FE130E04FEF64
:107AA0005FEF6DE770E088E290E00E949905109228
:107AB0003C064EE150E06AE471E015C09BE8E92E17
:107AC00094E0F92E02E02FE130E04FEF5FEF6DE739
:107AD00070E088E290E00E949905C0933C064EE178
:107AE00050E06CE271E083E096E00E94CA4780912A
:107AF0005206811110C0A895C0935F0610923E06F1
:107B000010923D06C0934D068FE190E00E94190649
:107B1000A8950E94DD1F80915206813059F5A895E5
:107B200080935F0610923E0610923D0680934D06AC
:107B30008FE190E00E9419061092970680913C0612
:107B4000813069F038F0823091F44EE150E06EE01F
:107B500071E009C04EE150E06AE471E004C04EE11A
:107B600050E06CE271E083E096E00E94CA47A8957D
:107B70000E941127D09352062FEF80E792E0215008
:107B800080409040E1F700C000001DCFDF91CF9111
:107B90001F910F91FF90EF900895EF92FF920F9336
:107BA0001F93CF93DF93A89580915F068111F6C054
:107BB0008FE190E00E9419060E944F0C809194067C
:107BC00090E0909338068093370685E080935206C4
:107BD000C1E0D5E080915F068111E0C0A8950E94C8
:107BE000DD0C809152068230A9F480913706909185
:107BF0003806019690933806809337060FE110E01F
:107C00002CE330E046EE50E069E670E081E090E081
:107C10000E94A404809152068330A9F48091370613
:107C200090913806019790933806809337060FE1BC
:107C300010E02CE330E046EE50E069E670E081E0D1
:107C400090E00E94A4048091370690913806039733
:107C500020F01092380610923706809137069091E6
:107C600038068130910589F1D0F0029709F046C0BD
:107C700081E8E82E84E0F82E02E02FE130E04FEFBB
:107C80005FEF6DE770E088E290E00E94990582E086
:107C9000809394064EE150E064EB70E02BC025E940
:107CA000E22E24E0F22E02E02FE130E04FEF5FEF12
:107CB0006DE770E088E290E00E94990510929406CA
:107CC0004EE150E060EF70E015C09BE8E92E94E0D3
:107CD000F92E02E02FE130E04FEF5FEF6DE770E04B
:107CE00088E290E00E949905C09394064EE150E02E
:107CF00062ED70E083E096E00E94CA4780915206F0
:107D0000811110C0A895C0935F0610923E06109294
:107D10003D06C0934D068FE190E00E941906A8959C
:107D20000E94DD1F80915206813061F5A8958093F5
:107D30005F0610923E0610923D0680934D068FE13D
:107D400090E00E941906A8951092970680919406DB
:107D5000813069F038F0823091F44EE150E064EB0C
:107D600070E009C04EE150E060EF70E004C04EE109
:107D700050E062ED70E083E096E00E94CA47A8956B
:107D80000E941127D09352062FEF80E792E02150F6
:107D900080409040E1F700C000001CCFDF91CF9100
:107DA0001F910F91FF90EF9008950F931F93809173
:107DB0002A0690912B06892B09F09EC080918B0694
:107DC00090918C0683359105A9F581E090E0909320
:107DD0002B0680932A060E9429140FE110E02CE361
:107DE00030E044E650E06BE470E08EE690E00E9404
:107DF000A40424E230E04AE550E064E670E088E064
:107E000090E00E94A40424E230E04AE550E064E6F9
:107E100070E088E090E00E94A40424E230E04AE5AB
:107E200050E064E670E08FED90E00E94A4040E94B0
:107E3000DD1FA8950E94B21E0E94931AA89503E028
:107E40002FE130E04FEF5FEF69E170E085E890E00F
:107E50000E9404110E94601E0E949C1080912A06BC
:107E600090912B060197A9F5A8950E9429140FE17E
:107E700010E02CE330E044E650E06BE470E08EE686
:107E800090E00E94A40424E230E04AE550E064E679
:107E900070E088E090E00E94A40424E230E04AE52B
:107EA00050E064E670E088E090E00E94A40424E2E0
:107EB00030E04AE550E064E670E08FED90E00E942B
:107EC000A4048091F105813009F4D0D10E94DD1F16
:107ED000A8952FEF81EE94E0215080409040E1F78B
:107EE00000C000000E94D20E0E94891E0E94580FFE
:107EF0001F910F910C94C80F1F910F9108951F921D
:107F00000F920FB60F9211248F939F938CB190E034
:107F100090938C0680938B069F918F910F900FBE4C
:107F20000F901F9018951F920F920FB60F92112469
:107F30002F938F939F938091FD059091FE0501965D
:107F4000883E23E0920728F49093FE058093FD0578
:107F500004C01092FE051092FD0580912806811143
:107F600005C010928E0610928D060BC0813049F428
:107F700080918D0690918E06019690938E06809347
:107F80008D0680914706811105C01092FC05109264
:107F9000FB050BC0813049F48091FB059091FC05F5
:107FA00001969093FC058093FB0580913F0681111B
:107FB00005C0109200061092FF050BC0813049F4F5
:107FC0008091FF05909100060196909300068093A2
:107FD000FF059F918F912F910F900FBE0F901F90D3
:107FE00018952FEF89E698E1215080409040E1F705
:107FF00000C000008FEF8ABB81BB8093610081E0ED
:1080000084BB88EA8FBD8CE08EBD1DBC1CBC17BC38
:1080100016BC8AE78BBD82E18ABD19BC18BC1092E0
:1080200079001092780080E187BF10BE87E683BF99
:1080300012BE11BE81E880938B0085E080938A0098
:108040001092890010928800109281001092800096
:108050001092870010928600109285001092840082
:1080600010928300109282001BB888E98AB986E0DA
:1080700080939500109290008FE289B98FE181BDC5
:108080008FE081BDCCD281E00E94B0038FE190E00F
:108090000E94190681E090E090932B0680932A06B7
:1080A00010923E0610923D0610922D0610922C065C
:1080B0001092FE051092FD051092440610924306A0
:1080C0001092FA051092290610928F06109222063D
:1080D00080E590E090938C0680938B0680916400FD
:1080E0008E7F80936400809165008160809365003D
:1080F000809164008860809364008091650088604E
:10810000809365001092F1057894A49AAC9A2FEFB1
:1081100085EA9EE0215080409040E1F700C00000D9
:10812000A895AC9882EB92E045D7813079F00E9417
:10813000D21AA8950E943F1EA89561E083EB92E0B9
:108140004FD7A89561E082EB92E04AD7A89580913D
:108150002A0690912B06019721F4A8950E94DD1F15
:10816000A895A89522DEF2CF80916400806180936B
:108170006400809165008061809365008091640057
:1081800088608093640080916500877F809365009C
:108190008091EC059091ED05893C910500F5809169
:1081A00064008460809364008091650084608093A3
:1081B00065008FEC97E00197F1F700C00000A895EB
:1081C000809165008B7F809365008091EC05909194
:1081D000ED0501969093ED058093EC05D9CF809144
:1081E00065008860809365000895809164008061D7
:1081F00080936400809165008F7E809365008091FC
:10820000640088608093640080916500877F80931C
:1082100065008091EC059091ED05893C910500F594
:108220008091640084608093640080916500846024
:10823000809365008FEC97E00197F1F700C0000094
:10824000A895809165008B7F809365008091EC05F7
:108250009091ED0501969093ED058093EC05D9CFB3
:108260008091650088608093650008958AEB92E0B4
:10827000A1D6809399068091640080618093640008
:1082800080916500806180936500809164008860C2
:108290008093640080916500877F80936500809162
:1082A000990628EC829FC00111242091EA053091A3
:1082B000EB052817390700F58091640084608093EE
:1082C0006400809165008460809365008FEC97E086
:1082D0000197F1F700C00000A895809165008B7FA1
:1082E000809365008091EA059091EB05019690934B
:1082F000EB058093EA05D3CF809165008860809379
:1083000065001092F0051092EB051092EA050895B1
:10831000AC018091F00581114AC090916400906198
:1083200090936400909165009F7E9093650090917A
:10833000640098609093640090916500977F90939B
:10834000650088EC849F9001859F300D11248091F9
:10835000EA059091EB058217930700F58091640080
:1083600084608093640080916500846080936500E0
:108370008FEC97E00197F1F700C00000A89580917D
:1083800065008B7F809365008091EA059091EB05F5
:1083900001969093EB058093EA05D9CF8091650013
:1083A0008860809365001092EB051092EA0581E0E9
:1083B0008093F0050895682F8AEB92E011C68AEB4E
:1083C00092E0F8D590E0A4CF8093EF050895CF9385
:1083D000DF9300D000D0CDB7DEB7809163001C8260
:1083E0001B821A821982BE016F5F7F4FCE010396F6
:1083F00029D18B819C818431954068F489819A814F
:10840000843A964040F489819A818D32914018F0E7
:1084100082E080939B068B819C818937954090F008
:108420008B819C81843C994068F489819A81843A4B
:10843000964040F489819A818D32914018F083E012
:1084400080939B068B819C8189329A4068F0898158
:108450009A8184379E4040F489819A81813D97407A
:1084600018F081E080939B068B819C81863F994028
:1084700060F48B819C818134964038F089819A81A7
:10848000813D974010F010929B0680919B060F90C3
:108490000F900F900F90DF91CF910895DF92EF92A0
:1084A000FF920F931F93CF93DF9385E080939B06FA
:1084B000DBE485E0D82E8091EF0581116FC087DF66
:1084C000E090EE05F12C03E02FE130E040E058EFC2
:1084D00062E870E080E590E00E94DF0580919B06F5
:1084E0008230B1F48091EE0581508093EE051092B8
:1084F000ED051092EC050FE110E02CE330E046EEC4
:1085000050E069E670E081E090E00E94A4042CDE77
:1085100080919B068330C1F48091EE058B34A0F4EA
:108520008F5F8093EE051092ED051092EC050FE140
:1085300010E02CE330E046EE50E069E670E081E0C8
:1085400090E00E94A40451DE8091EE058C3410F07E
:10855000D093EE0580919B0681110EC00FE110E0D3
:108560002CE330E046EE50E069E670E081E090E018
:108570000E94A4041092EE05C0919B06C13059F4EC
:108580008091EE0518DF8091EE0590E06FDE10928D
:10859000EE05C093EF05D0929B068DCFDF91CF9172
:1085A0001F910F91FF90EF90DF900895EF92FF924F
:1085B0000F938AEB92E0FED4E82EF12C03E02FE13A
:1085C00030E04FEF5FEF6AEA70E080EF90E00E94EA
:1085D000DF058AEB92E0EED480939A060F91FF902C
:1085E000EF900895EF92FF920F93E0909A06F12C8E
:1085F00003E02FE130E04FEF5FEF6AEA70E080EFD9
:1086000090E00E94DF050F91FF90EF900895C098D1
:10861000AB9AAF9A8FB9779BFECF8FB1089587E061
:1086200087BBC09AAB9AAF9A83E58DB91EB880E834
:10863000EEDF80E0ECDF80E0EADF8AE18A95F1F7A7
:1086400000C00895EF92FF920F931F93CF93DF9393
:1086500000D000D0CDB7DEB77C018B01A895AB9AD6
:10866000AF9A1C821B821A82198280EDD0DF80E0D3
:10867000CEDF8FB190E09C838B838B819C81982F80
:1086800088279C838B8380E0C2DF2FB18B819C8104
:10869000822B9C838B838B819C8133E0969587957D
:1086A0003A95E1F79C838B8387EC90E00197F1F793
:1086B00000C0000080E9ABDF80E0A9DF8FB190E06F
:1086C0009A83898389819A81982F88279A838983BD
:1086D00080E09DDF2FB189819A81822B9A838983E3
:1086E00089819A8153E0969587955A95E1F79A8307
:1086F00089838B819C81F7019183808389819A8111
:10870000F801918380830F900F900F900F90DF916D
:10871000CF911F910F91FF90EF90089570D088F046
:108720009F5790F0B92F9927B751A0F0D1F0660F5D
:10873000771F881F991F1AF0BA95C9F712C0B13078
:1087400081F077D0B1E0089574C0672F782F882723
:10875000B85F39F0B93FCCF3869577956795B395B7
:10876000D9F73EF490958095709561957F4F8F4F26
:108770009F4F0895E89409C097FB3EF4909580952B
:10878000709561957F4F8F4F9F4F9923A9F0F92FD7
:1087900096E9BB279395F695879577956795B79555
:1087A000F111F8CFFAF4BB0F11F460FF1BC06F5F3B
:1087B0007F4F8F4F9F4F16C0882311F096E911C04D
:1087C000772321F09EE8872F762F05C0662371F06E
:1087D00096E8862F70E060E02AF09A95660F771F82
:1087E000881FDAF7880F9695879597F9089557FDB2
:1087F0009058440F551F59F05F3F71F04795880F0F
:1088000097FB991F61F09F3F79F0879508951216A5
:1088100013061406551FF2CF4695F1DF08C0161651
:1088200017061806991FF1CF869571056105089402
:108830000895E894BB2766277727CB0197F9089519
:108840000BD078C069D028F06ED018F0952309F0CD
:108850005AC05FC01124EECFCADFA0F3959FD1F3B9
:10886000950F50E0551F629FF001729FBB27F00DDE
:10887000B11D639FAA27F00DB11DAA1F649F662733
:10888000B00DA11D661F829F2227B00DA11D621F82
:10889000739FB00DA11D621F839FA00D611D221F3C
:1088A000749F3327A00D611D231F849F600D211D20
:1088B000822F762F6A2F11249F5750408AF0E1F0C3
:1088C00088234AF0EE0FFF1FBB1F661F771F881F0C
:1088D00091505040A9F79E3F510570F014C0AACFA7
:1088E0005F3FECF3983EDCF3869577956795B795F7
:1088F000F795E7959F5FC1F7FE2B880F911D969521
:10890000879597F9089597F99F6780E870E060E090
:1089100008959FEF80EC089500240A941616170618
:1089200018060906089500240A9412161306140660
:1089300005060895092E0394000C11F4882352F0C3
:10894000BB0F40F4BF2B11F460FF04C06F5F7F4F7B
:108950008F4F9F4F0895AA1BBB1B51E107C0AA1F51
:10896000BB1FA617B70710F0A61BB70B881F991FD0
:108970005A95A9F780959095BC01CD010895EE0F09
:10898000FF1F0024001C0BBE0790F691E02D0994F8
:10899000A29FB001B39FC001A39F700D811D112440
:1089A000911DB29F700D811D1124911D0895BB274B
:1089B0004A3031F4992322F4BDE2909581959F4F7E
:1089C00001C0BB27FB015527AA27880F991FAA1FA3
:1089D000A41710F0A41B83955051B9F7A05DAA33DA
:1089E00008F0A95DA193009779F7B111B1931192A5
:1089F000CB0126C2CF93DF93CDB7DEB7AE014B5F7D
:108A00005F4FFA0161917191AF0180919E06909143
:108A10009F0603D0DF91CF9108952F923F924F92FE
:108A20005F926F927F928F929F92AF92BF92CF92FE
:108A3000DF92EF92FF920F931F93CF93DF93CDB707
:108A4000DEB72B970FB6F894DEBF0FBECDBF6C011B
:108A50007B018A01FC0117821682838181FFBFC1DD
:108A6000CE0101963C01F6019381F70193FD8591BA
:108A700093FF81917F01882309F4ADC1853239F4D8
:108A800093FD859193FF81917F01853221F4B60199
:108A900090E0E6D1E8CF912C212C312CFFE1F315A9
:108AA000D8F08B3279F038F4803279F08332A1F447
:108AB000232D20611DC08D3261F0803369F4232D98
:108AC000216016C0832D8260382EE32DE4603E2E97
:108AD0002AC0F32DF8601DC037FC2DC020ED280FF3
:108AE0002A3040F08E32B9F436FC75C1232D206453
:108AF000322E19C036FE06C08AE0989E200D112441
:108B0000922E11C0EAE02E9E200D1124222EF32D6C
:108B1000F0623F2E08C08C3621F4832D8068382EF9
:108B200002C0883641F4F70193FD859193FF81914E
:108B30007F018111B3CF982F9F7D9554933028F4F6
:108B40000C5F1F4F9FE399830DC0833631F083374D
:108B500071F0833509F055C020C0F8018081898308
:108B60000E5F1F4F88248394912C530112C028015B
:108B7000F2E04F0E511CF801A080B18036FE03C018
:108B8000692D70E002C06FEF7FEFC5014ED14C013F
:108B90008201F32DFF773F2E15C0280122E0420EFF
:108BA000511CF801A080B18036FE03C0692D70E031
:108BB00002C06FEF7FEFC5012DD14C01F32DF0689E
:108BC0003F2E820133FC19C0822D90E08816990651
:108BD000A0F4B60180E290E043D12A94F5CFF501EC
:108BE00037FC859137FE81915F01B60190E038D165
:108BF00021102A9421E0821A91088114910479F7B6
:108C0000E1C0843611F0893639F5F80137FE07C026
:108C100060817181828193810C5F1F4F08C06081E8
:108C20007181072E000C880B990B0E5F1F4FF32DDF
:108C3000FF763F2E97FF09C09095809570956195BE
:108C40007F4F8F4F9F4FF0683F2E2AE030E0A30107
:108C500043D1882E861844C0853731F4232D2F7ECA
:108C6000B22E2AE030E025C0932D997FB92E8F36A1
:108C7000C1F018F4883579F0AEC0803719F0883724
:108C800021F0A9C0E92FE061BE2EB4FE0DC0FB2D7E
:108C9000F460BF2E09C034FE0AC0292F2660B22E10
:108CA00006C028E030E005C020E130E002C020E14D
:108CB00032E0F801B7FE07C0608171818281938143
:108CC0000C5F1F4F06C06081718180E090E00E5FF5
:108CD0001F4FA30101D1882E8618FB2DFF773F2E51
:108CE00036FE0DC0232D2E7FA22E891458F434FE9B
:108CF0000BC032FC09C0832D8E7EA82E05C0B82C77
:108D0000A32C03C0B82C01C0B92CA4FE0FC0FE01D7
:108D1000E80DF11D8081803321F49A2D997EA92ED2
:108D200009C0A2FE06C0B394B39404C08A2D86780D
:108D300009F0B394A3FC10C0A0FE06C0B21480F4E6
:108D4000280C922C9B180DC0B21458F4B60180E286
:108D500090E086D0B394F8CFB21418F42B1802C068
:108D6000982C212CA4FE0FC0B60180E390E078D0AF
:108D7000A2FE16C0A1FC03C088E790E002C088E50F
:108D800090E0B6010CC08A2D867851F0A1FE02C099
:108D90008BE201C080E2A7FC8DE2B60190E060D0DA
:108DA000891430F4B60180E390E05AD09A94F8CF59
:108DB0008A94F301E80DF11D8081B60190E050D056
:108DC0008110F6CF222009F44ECEB60180E290E069
:108DD00047D02A94F7CFF6018681978102C08FEFA2
:108DE0009FEF2B960FB6F894DEBF0FBECDBFDF917D
:108DF000CF911F910F91FF90EF90DF90CF90BF9098
:108E0000AF909F908F907F906F905F904F903F902A
:108E10002F900895FC010590615070400110D8F723
:108E2000809590958E0F9F1F0895FC0161507040B2
:108E300001900110D8F7809590958E0F9F1F08958F
:108E4000DC01FC01672F71917723E1F7329704C0B1
:108E50007C916D9370836291AE17BF07C8F308953C
:108E60000F931F93CF93DF93FB01238121FD03C059
:108E70008FEF9FEF2CC022FF16C0468157812481BF
:108E800035814217530744F4A081B1819D012F5FC2
:108E90003F4F318320838C93268137812F5F3F4F53
:108EA0003783268314C08B01EC01FB010084F1851C
:108EB000E02D0995892BE1F6D80116968D919C91AC
:108EC0001797019617969C938E931697CE01DF9174
:108ED000CF911F910F910895FA01AA27283051F1DF
:108EE000203181F1E8946F936E7F6E5F7F4F8F4FDB
:108EF0009F4FAF4FB1E03ED0B4E03CD0670F781F3A
:108F0000891F9A1FA11D680F791F8A1F911DA11D1E
:108F10006A0F711D811D911DA11D20D009F4689457
:108F20003F912AE0269F11243019305D3193DEF6FF
:108F3000CF010895462F4770405D4193B3E00FD0B5
:108F4000C9F7F6CF462F4F70405D4A3318F0495DA0
:108F500031FD4052419302D0A9F7EACFB4E0A69583
:108F60009795879577956795BA95C9F700976105A5
:108F7000710508959B01AC010A2E069457954795FB
:108F800037952795BA95C9F7620F731F841F951FF0
:108F9000A01D0895DC01CB01FC01E199FECF06C0C4
:108FA000FFBBEEBBE09A31960DB20D92415050409E
:108FB000B8F70895E199FECF9FBB8EBBE09A992741
:108FC0008DB30895A8E1B0E042E050E0E5CFDC01C8
:108FD000CB0102C02D9105D041505040D8F70895E3
:108FE000262FE199FECF9FBB8EBB2DBB0FB6F89409
:108FF000E29AE19A0FBE01960895F2DF272FF1CF92
:04900000F894FFCF12
:109004000000000200000000DE07000000005754CA
:109014003D2025750A47530047533D2025750A53C3
:109024004E00534E3D2025750A454E4400574B3D96
:109034002025750A565000503D332E360A520052F0
:109044004C3D2025750A68004F3D73740A53004750
:109054003D73740A530053523D53746174696F6EC7
:10906400200A57500057503D536E36332F50623309
:10907400370A57540057503D536E41670A575400FE
:1090840057503D50726F66696C65300A57540057EB
:10909400503D50726F66696C65310A5754005750E1
:1090A4003D50726F66696C65320A57540057503DE3
:1090B40050726F66696C65330A57540057503D50BF
:1090C400726F66696C65340A57540057503D50728C
:1090D4006F66696C65350A57540053523D555068A4
:1090E4006561746572200A57500053523D50726591
:1090F400686561746572200A57500053523D4D6192
:109104006E75616C200A57500053523D5265626F70
:109114006C6C696E67200A57500053523D4368696E
:109124007068656174696E67200A57500053523D38
:1091340050434268656174696E67200A5750005352
:10914400523D5043200A575000C2FBE1E5F0E8F2DB
:10915400E520E2FBF1EEF2F30056312E327A0020E4
:109164002020C2F0E5ECFF20F0E5E1EEEBEBE8EDCA
:10917400E3E02020202000C2FBE1E5F0E8F2E52056
:10918400F0E5E6E8EC00D2E5ECEFE5F0E0F2F3F030
:10919400E020EFEEEBEEF7EAE8202000EDE8E7E070
:1091A40020EFF0E820E4EEEDE0E3F0E5E2E500D2C4
:1091B400E5ECEFE5F0E0F2F3F0E020F3E2E5EBE8D4
:1091C400F7E5EDE8FF00202020202020E4EEEDE08C
:1091D400E3F0E5E2E020202020202000C4EBE8F2C8
:1091E400E5EBFCEDEEF1F2FC20E2EFE8F2FBE2E06D
:1091F400EDE8FF00D4F3EDEAF6E8FF20E4EEEDEE4F
:10920400E3F0E5E2E000EDE8E6EDE5E3EE20EDE095
:10921400E3F0E5E2E0F2E5EBFF2020202000CCE0E3
:10922400EAF1E8ECE0EBFCEDE0FF20ECEEF9EDEE2A
:10923400F1F2FC202000E2E5F0F5EDE5E3EE20EDAF
:10924400E0E3F0E5E2E0F2E5EBFF20202000CCE0F3
:10925400EAF1E8ECE0EBFCEDE0FF20ECEEF9EDEEFA
:10926400F1F2FC202000E2E5F0F5EDE5E3EE20ED7F
:10927400E0E3F0E5E2E0F2E5EBFF20202000D2E5B8
:10928400ECEFE5F0E0F2F3F0E020E2EAEBFEF7E5E4
:10929400EDE8FF202000CAEEEDF2F0EEEBFC20EF4B
:1092A400EE20E2E5F0F5F320202020202000EDE878
:1092B400E6EDE5E3EE20EDE0E3F0E5E2E0F2E5EBF8
:1092C400FF2020202000CAEEFDF4F4E8F6E8E5EDE6
:1092D400F220EFF0EEF4E8EBFF2020202000E2E59E
:1092E400F0F5EDE5E3EE20EDE0E3F0E5E2E0F2E5B4
:1092F400EBFF20202000CAEEFDF4F4E8F6E8E5EDEB
:10930400F220EFF0EEF4E8EBFF2020202000EDE067
:10931400E3F0E5E2E0F2E5EBFF202000D2E5ECEF3C
:10932400E5F0E0F2F3F0E020EDE8E6EDE5E3EE2031
:1093340020202000EFE0E9EAE82000D2E5ECEFE5A8
:10934400F0E0F2F3F0E020ECE5F1F2E02020202060
:109354002000C2FBE1E5F0E8F2E520EFF0EEF4E8EE
:10936400EBFC00CFF0EEF4E8EBFC203500CFF0EEA0
:10937400F4E8EBFC203400CFF0EEF4E8EBFC20330F
:1093840000CFF0EEF4E8EBFC203200CFF0EEF4E88E
:10939400EBFC203100CFF0EEF4E8EBFC203000537E
:1093A4006E416700536E506200CAEEECEFFCFEF2B1
:1093B400E5F000C4EEEF2E20EDE0F1F2F0EEE9EA84
:1093C400E800EFEBE0F20020D1F3F8EAE020EFEB65
:1093D400E0F22000ECE8EAF0EEF1F5E5EC00D1F380
:1093E400F8EAE000D0E5E1EEEBEBE8EDE32000D0B5
:1093F400F3F7EDEEE9002020D0F3F7EDEEE92020BD
:109404002000CDE8E6EDE8E920EDE0E3F02E2000D1
:10941400C2E5F0F5EDE8E920EDE0E3F02E002020D0
:10942400D1F2E0EDF6E8FF00E2E5F0F5E000EDE86A
:10943400E7E000CCEEF9EDEEF1F2FC00CFF0E8ED60
:10944400FFF2EE202000C2DBC1D0C0D2DC00C2DBC0
:10945400CACB00C2CACB00CDE0F1F2F0EEE8F2FCD8
:1094640000C7E2F3EAEEE2FBE520F1E8E3EDE0EB2E
:10947400FB00CFF0E5E4F3F1F2E0EDEEE2EAE80020
:10948400D3ECEEEBF7E0EDE8FF00C2F0E5ECFF20F3
:10949400EFE0E9EAE80020C4E0F2F7E8EA20EDE8CA
:1094A400E62E20EDE0E3F0E5E2E0F2E5EBFF00205C
:1094B400C4E0F2F7E8EA20ECE5F1F2E020EFE0E9BD
:1094C400EAE800F0F3F7EDEEE900EDE8E6EDE8E9AF
:1094D40000EDE0E3F02E00C2E5F0F5EDE8E900C2AE
:0694E400DBD5CEC4000040
:00000001FF
